:020000040800F2
:100000008C010020BD020008D1020008D3020008C4
:10001000D5020008D7020008D9020008000000003D
:10002000000000000000000000000000DB020008EB
:10003000DD02000800000000DF020008E102000805
:10004000E3020008E5020008E7020008E9020008F0
:10005000EB020008ED020008EF020008F1020008C0
:10006000F3020008F5020008F7020008F902000890
:10007000FB020008411A0208FF0200080103000801
:10008000030300080503000807030008090300082C
:100090000B0300080D0300080F03000811030008FC
:1000A000D150020811510208170300081903000873
:1000B0001B0300085950020895500208210300084C
:1000C000230300082503000827030008290300086C
:1000D0002B0300082D0300082F030008310300083C
:1000E000330300083503000837030008390300080C
:1000F0003B0300083D0300083F03000841030008DC
:1001000043030008450300089B5102084903000807
:100110004B0300084D0300084F030008615102081B
:10012000530300085503000857030008634E0208F4
:100130005B0300085D0300085F030008610300081B
:1001400063030008650300086703000869030008EB
:100150006B0300086D0300086F03000871030008BB
:10016000730300087503000877030008790300088B
:100170007B0300087D0300087F030008810300085B
:10018000830300088503000887030008890300082B
:100190008B0300088D0300088F03000891030008FB
:0C01A00093030008950300089703000873
:1001AC002A49072291438D4629482A492A4A00F0B8
:1001BC003AF82A482A492B4A00F035F82A482B49A4
:1001CC002B4A00F030F82B482B492C4A00F02BF826
:1001DC002B482C492C4A00F026F82C482C492D4A47
:1001EC0000F021F82C482D49002200F027F82C486B
:1001FC002C49091A082903DB002202600430016033
:10020C001D481E49884205D00268043003B490474B
:10021C0003BCF7E700208646EC4600200021BBE03B
:10022C00214A9047FEE7884207D0521A05D003783E
:10023C0001300B700131013AF9D17047884202D07C
:10024C0002700130FAE77047184870478C010020A3
:10025C00D05E02080000002000000020A40300086B
:10026C00A4030008B05E0208D05E02080000002063
:10027C0000000020B05E0208B05E0208B05E02080A
:10028C00B05E0208B05E0208B05E0208B05E020802
:10029C00B05E0208D05E0208000000200C000020B6
:1002AC000C0000208C000020A4030008FFFFFFFFBF
:1002BC003648854600F005F8354836490160FFF7A9
:1002CC006FBF7047FEE7FEE7FEE7FEE7FEE7FEE7DF
:1002DC00FEE7FEE7FEE7FEE7FEE7FEE7FEE7FEE7EA
:1002EC00FEE7FEE7FEE7FEE7FEE7FEE7FEE7FEE7DA
:1002FC00FEE7FEE7FEE7FEE7FEE7FEE7FEE7FEE7CA
:10030C00FEE7FEE7FEE7FEE7FEE7FEE7FEE7FEE7B9
:10031C00FEE7FEE7FEE7FEE7FEE7FEE7FEE7FEE7A9
:10032C00FEE7FEE7FEE7FEE7FEE7FEE7FEE7FEE799
:10033C00FEE7FEE7FEE7FEE7FEE7FEE7FEE7FEE789
:10034C00FEE7FEE7FEE7FEE7FEE7FEE7FEE7FEE779
:10035C00FEE7FEE7FEE7FEE7FEE7FEE7FEE7FEE769
:10036C00FEE7FEE7FEE7FEE7FEE7FEE7FEE7FEE759
:10037C00FEE7FEE7FEE7FEE7FEE7FEE7FEE7FEE749
:10038C00FEE7FEE7FEE7FEE7FEE7FEE700000320E0
:08039C0008ED00E0000000087C
:1003A40003F02CBE0000000000000000000000006C
:1003B4000000000000000000000000000000000039
:1003C4000000000000000000000000000000000029
:1003D4000000000000000000000000000000000019
:1003E4000000000000000000000000000000000009
:103FF4000000000000000000000000000BF0FEBF05
:1040040000000000000000000000000000000000AC
:10401400000000000000000000000000000000009C
:10402400000000000000000000000000000000008C
:10403400000000000000000000000000000000007C
:020000040801F1
:100000004FF000506FF00006C0F8E464C0F8E465FB
:10001000C0F8E466C0F8E467C0F8E468C0F8E469D2
:10002000C0F8E46AC0F8E46B40F60000C4F20000D7
:1000300040F20101C0F20001C16040F20101C0F2D2
:100040000001816240F2DC6140F26E31C16240F237
:100050008501C0F20001016040F20101C0F200011F
:10006000416140F20040C4F2000040F20101C0F2E0
:100070000001C16040F20101C0F20001816240F262
:100080006E31C16240F28501C0F20001016040F2B0
:100090000101C0F20001416140F20000C4F2010020
:1000A00040F20101C0F20001C16040F20101C0F262
:1000B0000001816240F26E31C16240F28501C0F2FE
:1000C0000001016040F20101C0F20001416144F20F
:1000D0000000C4F2010040F20101C0F20001C16061
:1000E00040F20101C0F20001816240F26E31C16252
:1000F00040F28501C0F20001016040F20101C0F24E
:100100000001416141F20040C4F2000040F20101EF
:10011000C0F20001C16040F20001C0F20001816242
:1001200042F22831C16240F28501C0F2000140F282
:100130000101C0F2000140F60040C4F2000040F2AC
:100140000101C0F20001C16040F2000181624FF67E
:10015000FF71C16240F28501C0F2000140F201016D
:10016000C0F200014EF20010CEF20000016842F22F
:100170000002C7F2007241EA02010160416840F2E8
:100180002002C0F6941241EA02014160816840F207
:100190000002C0F2000241EA020143F20043C4F24D
:1001A000010341F20004C4F202044FF00001C0F266
:1001B0001001A16140F21001197300BF00BF00BF20
:1001C00000BF198911F00201FBD0198911F08001DB
:1001D000FBD140F21001A161998900BF00BF00BFAF
:1001E00000BF40F220310139FDD143F20043C4F297
:1001F000010341F20004C4F202044FF00001C0F216
:100200001001A16140F26401197300BF00BF00BF7B
:1002100000BF198911F00201FBD0198911F080018A
:10022000FBD140F21001A161998900BF00BF00BF5E
:1002300000BF43F60003C4F2000340F20044C4F2DE
:10024000020440F60045C4F202054FF00001C1F27D
:100250000001A1614FF00001C0F24001A96140F22C
:100260000601197300BF00BF00BF00BF198911F05C
:100270000201FBD0198911F08001FBD141F200018C
:10028000A16140F24001A961197B00BF00BF00BF1E
:1002900000BF4FF00001C1F20001A1614FF0000169
:1002A000C0F24001A96140F20101197300BF00BF13
:1002B00000BF00BF198911F00201FBD0198911F0AC
:1002C0008001FBD1197B40F20201197300BF00BF0E
:1002D00000BF00BF198911F00201FBD0198911F08C
:1002E0008001FBD141F20001A16140F24001A9610E
:1002F000197B00BF00BF00BF00BF4FF000504FF0A0
:100300000001C1F20001A1614FF00001C0F2400103
:10031000A96140F20301197300BF00BF00BF00BF15
:10032000198911F00201FBD0198911F08001FBD16C
:10033000197B40F20001197300BF00BF00BF00BF6E
:10034000198911F00201FBD0198911F08001FBD14C
:10035000197B00BF00BF00BF00BF40F2000119734E
:1003600000BF00BF00BF00BF198911F00201FBD020
:10037000198911F08001FBD1197B00BF00BF00BFBC
:1003800000BF40F20001197300BF00BF00BF00BFF3
:10039000198911F00201FBD0198911F08001FBD1FC
:1003A000197B00BF00BF00BF00BF40F200011973FE
:1003B00000BF00BF00BF00BF198911F00201FBD0D0
:1003C000198911F08001FBD1197BA92940F0B08077
:1003D00000BF00BF40F20001197300BF00BF00BFA3
:1003E00000BF198911F00201FBD0198911F08001B9
:1003F000FBD1197BA92940F09B8000BF00BF40F2D0
:100400000001197300BF00BF00BF00BF198911F0C0
:100410000201FBD0198911F08001FBD1197BA929B8
:1004200040F0868000BF00BF40F20001197300BF9A
:1004300000BF00BF00BF198911F00201FBD019896C
:1004400011F08001FBD1197BA92971D100BF00BF38
:1004500040F20001197300BF00BF00BF00BF19893F
:1004600011F00201FBD0198911F08001FBD11E7B34
:1004700006F0FF064FEA062600BF00BF40F200016B
:10048000197300BF00BF00BF00BF198911F002013E
:10049000FBD0198911F08001FBD1197B01F0FF011C
:1004A00046EA010640F2FF3106EA0106A0F8FC6EBA
:1004B000A0F8546000BF00BF40F20001197300BFF4
:1004C00000BF00BF00BF198911F00201FBD01989DC
:1004D00011F08001FBD1197B80F8211D80F8FA1EF4
:1004E00080F86A1000BF00BF00BF00BF40F20001EB
:1004F000197300BF00BF00BF00BF198911F00201CE
:10050000FBD0198911F08001FBD1197B80F8201DE7
:1005100080F8FB1E80F86B1000BF00BF00BF00BF5B
:1005200041F20001A16140F24001A9610FF068BDF4
:1005300041F20001A16140F24001A9614FF0005079
:100540004FF00001A0F8FC1EA0F8541080F8211D07
:1005500080F8FA1E80F86A104FF0500180F8201DD4
:1005600080F8FB1E80F86B1043F60003C4F2000312
:1005700040F20044C4F2020440F60045C4F2020511
:100580004FF00001C1F20001A1614FF00001C0F283
:100590004001A96140F20601197300BF00BF00BF0E
:1005A00000BF198911F00201FBD0198911F08001F7
:1005B000FBD141F20001A16140F24001A961197B28
:1005C00000BF00BF00BF00BF4FF00001C1F200013B
:1005D000A1614FF00001C0F24001A96140F20201A7
:1005E000197300BF00BF00BF00BF198911F00201DD
:1005F000FBD0198911F08001FBD1197B00BF00BF2E
:1006000000BF00BF40F20001197300BF00BF00BF70
:1006100000BF198911F00201FBD0198911F0800186
:10062000FBD1197B00BF00BF00BF00BF40F200013B
:10063000197300BF00BF00BF00BF198911F002018C
:10064000FBD0198911F08001FBD1197B00BF00BFDD
:1006500000BF00BF40F20001197300BF00BF00BF20
:1006600000BF198911F00201FBD0198911F0800136
:10067000FBD1197B00BF00BF00BF00BF4FF0A90135
:10068000197300BF00BF00BF00BF198911F002013C
:10069000FBD0198911F08001FBD1197B00BF00BF8D
:1006A00000BF00BF4FF0A901197300BF00BF00BF1A
:1006B00000BF198911F00201FBD0198911F08001E6
:1006C000FBD1197B00BF00BF00BF00BF4FF0A901E5
:1006D000197300BF00BF00BF00BF198911F00201EC
:1006E000FBD0198911F08001FBD1197B00BF00BF3D
:1006F00000BF00BF4FF0A901197300BF00BF00BFCA
:1007000000BF198911F00201FBD0198911F0800195
:10071000FBD1197B00BF00BF00BF00BFB0F8541071
:100720004FEA1121197300BF00BF00BF00BF198934
:1007300011F00201FBD0198911F08001FBD1197B66
:1007400000BF00BF00BF00BFB0F85410197300BF56
:1007500000BF00BF00BF198911F00201FBD0198949
:1007600011F08001FBD1197B00BF00BF00BF00BFAB
:100770004FF00001197300BF00BF00BF00BF19890F
:1007800011F00201FBD0198911F08001FBD1197B16
:1007900000BF00BF00BF00BF4FF05001197300BF82
:1007A00000BF00BF00BF198911F00201FBD01989F9
:1007B00011F08001FBD1197B00BF00BF00BF00BF5B
:1007C00041F20001A16140F24001A9610FF018BCA3
:1007D0000000000000000000000000000000000019
:1007E0000000000000000000000000000000000009
:1007F00000000000000000000000000000000000F9
:1008000000000000000000000000000000000000E8
:020000040802F0
:100000004FF00050017A21F00101017242F24C0AD6
:10001000C4F2010ABAF800604EF60001C2F2000113
:100020004EF60012C2F2000221F8026B9142FBD19F
:100030004FEAD606A0F8B0604FF0000181834FF080
:10004000005090F80C114FEA810141F0400180F816
:10005000F91EB0F85610B0F8FC2E914240F01D8207
:10006000B0F86810B0F85420914200F0BC80A0F8BD
:10007000541043F60003C4F2000340F20044C4F2FB
:10008000020440F60045C4F202054FF00001C1F23F
:100090000001A1614FF00001C0F24001A96140F2EE
:1000A0000601197300BF00BF00BF00BF198911F01E
:1000B0000201FBD0198911F08001FBD141F200014E
:1000C000A16140F24001A961197B00BF00BF00BFE0
:1000D00000BF4FF00001C1F20001A1614FF000012B
:1000E000C0F24001A96140F20201197300BF00BFD4
:1000F00000BF00BF198911F00201FBD0198911F06E
:100100008001FBD1197B00BF00BF00BF00BF40F2E0
:100110000001197300BF00BF00BF00BF198911F0B3
:100120000201FBD0198911F08001FBD1197B00BFBE
:1001300000BF00BF00BF40F20001197300BF00BF45
:1001400000BF00BF198911F00201FBD0198911F01D
:100150008001FBD1197B00BF00BF00BF00BF40F290
:100160000401197300BF00BF00BF00BF198911F05F
:100170000201FBD0198911F08001FBD1197B00BF6E
:1001800000BF00BF00BFB0F868104FEA112119731B
:1001900000BF00BF00BF00BF198911F00201FBD0F2
:1001A000198911F08001FBD1197B00BF00BF00BF8E
:1001B00000BFB0F86810197300BF00BF00BF00BFD8
:1001C000198911F00201FBD0198911F08001FBD1CE
:1001D000197B00BF00BF00BF00BF41F20001A16159
:1001E00040F24001A96190F8211D90F86A209142E7
:1001F00000F0A680A0F86A1043F60003C4F20003E2
:1002000040F20044C4F2020440F60045C4F2020584
:100210004FF00001C1F20001A1614FF00001C0F2F6
:100220004001A96140F20601197300BF00BF00BF81
:1002300000BF198911F00201FBD0198911F080016A
:10024000FBD141F20001A16140F24001A961197B9B
:1002500000BF00BF00BF00BF4FF00001C1F20001AE
:10026000A1614FF00001C0F24001A96140F202011A
:10027000197300BF00BF00BF00BF198911F0020150
:10028000FBD0198911F08001FBD1197B00BF00BFA1
:1002900000BF00BF40F20001197300BF00BF00BFE4
:1002A00000BF198911F00201FBD0198911F08001FA
:1002B000FBD1197B00BF00BF00BF00BF40F20001AF
:1002C000197300BF00BF00BF00BF198911F0020100
:1002D000FBD0198911F08001FBD1197B00BF00BF51
:1002E00000BF00BF40F20601197300BF00BF00BF8E
:1002F00000BF198911F00201FBD0198911F08001AA
:10030000FBD1197B00BF00BF00BF00BF90F8211DCB
:10031000197300BF00BF00BF00BF198911F00201AF
:10032000FBD0198911F08001FBD1197B00BF00BF00
:1003300000BF00BF41F20001A16140F24001A9618C
:1003400090F8201D90F86B20914200F0A680A0F854
:100350006B1043F60003C4F2000340F20044C4F201
:10036000020440F60045C4F202054FF00001C1F25C
:100370000001A1614FF00001C0F24001A96140F20B
:100380000601197300BF00BF00BF00BF198911F03B
:100390000201FBD0198911F08001FBD141F200016B
:1003A000A16140F24001A961197B00BF00BF00BFFD
:1003B00000BF4FF00001C1F20001A1614FF0000148
:1003C000C0F24001A96140F20201197300BF00BFF1
:1003D00000BF00BF198911F00201FBD0198911F08B
:1003E0008001FBD1197B00BF00BF00BF00BF40F2FE
:1003F0000001197300BF00BF00BF00BF198911F0D1
:100400000201FBD0198911F08001FBD1197B00BFDB
:1004100000BF00BF00BF40F20001197300BF00BF62
:1004200000BF00BF198911F00201FBD0198911F03A
:100430008001FBD1197B00BF00BF00BF00BF40F2AD
:100440000701197300BF00BF00BF00BF198911F079
:100450000201FBD0198911F08001FBD1197B00BF8B
:1004600000BF00BF00BF90F8201D197300BF00BF80
:1004700000BF00BF198911F00201FBD0198911F0EA
:100480008001FBD1197B00BF00BF00BF00BF41F25C
:100490000001A16140F24001A9614FF0005047F214
:1004A0000004C1F2000490F80A1D4FEA0161A16145
:1004B0006FEA0101E16190F8121D4FEA01612162CA
:1004C0004FEA516280F863246FEA0101616290F89B
:1004D000021D4FEA0161A1636FEA0101E16390F837
:1004E000501D4FEA016121646FEA0101616490F8D7
:1004F000511D4FEA0161A1646FEA0101E16490F8C6
:10050000521D4FEA016121656FEA0101616590F8B2
:10051000531D4FEA0161A1656FEA0101E16590F8A1
:10052000541D4FEA016121666FEA0101616690F88E
:10053000551D4FEA0161A1666FEA0101E16690F87D
:10054000561D4FEA016121676FEA0101616790F86A
:10055000571D4FEA0161A1676FEA0101E16790F859
:10056000581D4FEA0161C4F880106FEA0101C4F818
:10057000841090F8591D4FEA0161C4F888106FEAA1
:100580000101C4F88C1090F85A1D4FEA0161C4F8BB
:1005900090106FEA0101C4F8941090F85B1D4FEAC7
:1005A0000161C4F898106FEA0101C4F89C1090F83A
:1005B0005C1D4FEA0161C4F8A0106FEA0101C4F8A4
:1005C000A41090F85D1D4FEA0161C4F8A8106FEA0D
:1005D0000101C4F8AC1090F85E1D4FEA0161C4F847
:1005E000B0106FEA0101C4F8B41090F85F1D4FEA33
:1005F0000161C4F8B8106FEA0101C4F8BC1090F8AA
:10060000601D4FEA0161C4F8C0106FEA0101C4F82F
:10061000C41090F8611D4FEA0161C4F8C8106FEA78
:100620000101C4F8CC1090F8621D4FEA0161C4F8D2
:10063000D0106FEA0101C4F8D41090F8631D4FEA9E
:100640000161C4F8D8106FEA0101C4F8DC1004F5A8
:10065000807490F80B1D4FEA0161A1616FEA0101FE
:10066000E16190F8131D4FEA016121624FEA516286
:1006700080F863256FEA0101616290F8031D4FEA7B
:100680000161A1636FEA0101E16390F8701D4FEA17
:10069000016121646FEA0101616490F8711D4FEA04
:1006A0000161A1646FEA0101E16490F8721D4FEAF3
:1006B000016121656FEA0101616590F8731D4FEAE0
:1006C0000161A1656FEA0101E16590F8741D4FEACF
:1006D000016121666FEA0101616690F8751D4FEABC
:1006E0000161A1666FEA0101E16690F8761D4FEAAB
:1006F000016121676FEA0101616790F8771D4FEA98
:100700000161A1676FEA0101E16790F8781D4FEA86
:100710000161C4F880106FEA0101C4F8841090F8F8
:10072000791D4FEA0161C4F888106FEA0101C4F82D
:100730008C1090F87A1D4FEA0161C4F890106FEAAE
:100740000101C4F8941090F87B1D4FEA0161C4F8D0
:1007500098106FEA0101C4F89C1090F87C1D4FEAD4
:100760000161C4F8A0106FEA0101C4F8A41090F868
:100770007D1D4FEA0161C4F8A8106FEA0101C4F8B9
:10078000AC1090F87E1D4FEA0161C4F8B0106FEA1A
:100790000101C4F8B41090F87F1D4FEA0161C4F85C
:1007A000B8106FEA0101C4F8BC1090F8801D4FEA40
:1007B0000161C4F8C0106FEA0101C4F8C41090F8D8
:1007C000811D4FEA0161C4F8C8106FEA0101C4F845
:1007D000CC1090F8821D4FEA0161C4F8D0106FEA86
:1007E0000101C4F8D41090F8831D4FEA0161C4F8E8
:1007F000D8106FEA0101C4F8DC1004F5807490F899
:100800000C1D4FEA0161A1616FEA0101E16190F8FD
:10081000141D4FEA016121624FEA516280F863269C
:100820006FEA0101616290F8041D4FEA0161A16362
:100830006FEA0101E16390F8901D4FEA01612164C4
:100840006FEA0101616490F8911D4FEA0161A164B2
:100850006FEA0101E16490F8921D4FEA01612165A0
:100860006FEA0101616590F8931D4FEA0161A1658E
:100870006FEA0101E16590F8941D4FEA016121667C
:100880006FEA0101616690F8951D4FEA0161A1666A
:100890006FEA0101E16690F8961D4FEA0161216758
:1008A0006FEA0101616790F8971D4FEA0161A16746
:1008B0006FEA0101E16790F8981D4FEA0161C4F801
:1008C00080106FEA0101C4F8841090F8991D4FEA76
:1008D0000161C4F888106FEA0101C4F88C1090F827
:1008E0009A1D4FEA0161C4F890106FEA0101C4F843
:1008F000941090F89B1D4FEA0161C4F898106FEABC
:100900000101C4F89C1090F89C1D4FEA0161C4F8E5
:10091000A0106FEA0101C4F8A41090F89D1D4FEAE1
:100920000161C4F8A8106FEA0101C4F8AC1090F896
:100930009E1D4FEA0161C4F8B0106FEA0101C4F8CE
:10094000B41090F89F1D4FEA0161C4F8B8106FEA27
:100950000101C4F8BC1090F8A01D4FEA0161C4F871
:10096000C0106FEA0101C4F8C41090F8A11D4FEA4D
:100970000161C4F8C8106FEA0101C4F8CC1090F806
:10098000A21D4FEA0161C4F8D0106FEA0101C4F85A
:10099000D41090F8A31D4FEA0161C4F8D8106FEA93
:1009A0000101C4F8DC1004F5807490F80D1D4FEAC5
:1009B0000161A1616FEA0101E16190F8151D4FEA43
:1009C000016121624FEA516280F863276FEA0101F9
:1009D000616290F8051D4FEA0161A1636FEA0101B0
:1009E000E16390F8B01D4FEA016121646FEA0101F3
:1009F000616490F8B11D4FEA0161A1646FEA0101E1
:100A0000E16490F8B21D4FEA016121656FEA0101CE
:100A1000616590F8B31D4FEA0161A1656FEA0101BC
:100A2000E16590F8B41D4FEA016121666FEA0101AA
:100A3000616690F8B51D4FEA0161A1666FEA010198
:100A4000E16690F8B61D4FEA016121676FEA010186
:100A5000616790F8B71D4FEA0161A1676FEA010174
:100A6000E16790F8B81D4FEA0161C4F880106FEAA1
:100A70000101C4F8841090F8B91D4FEA0161C4F86F
:100A800088106FEA0101C4F88C1090F8BA1D4FEA83
:100A90000161C4F890106FEA0101C4F8941090F855
:100AA000BB1D4FEA0161C4F898106FEA0101C4F858
:100AB0009C1090F8BC1D4FEA0161C4F8A0106FEAC9
:100AC0000101C4F8A41090F8BD1D4FEA0161C4F8FB
:100AD000A8106FEA0101C4F8AC1090F8BE1D4FEAEF
:100AE0000161C4F8B0106FEA0101C4F8B41090F8C5
:100AF000BF1D4FEA0161C4F8B8106FEA0101C4F8E4
:100B0000BC1090F8C01D4FEA0161C4F8C0106FEA34
:100B10000101C4F8C41090F8C11D4FEA0161C4F886
:100B2000C8106FEA0101C4F8CC1090F8C21D4FEA5A
:100B30000161C4F8D0106FEA0101C4F8D41090F834
:100B4000C31D4FEA0161C4F8D8106FEA0101C4F86F
:100B5000DC1004F5807490F80E1D4FEA0161A1616C
:100B60006FEA0101E16190F8161D4FEA016121620F
:100B70004FEA516280F863286FEA0101616290F8E0
:100B8000061D4FEA0161A1636FEA0101E16390F87C
:100B9000D01D4FEA016121646FEA0101616490F8A0
:100BA000D11D4FEA0161A1646FEA0101E16490F88F
:100BB000D21D4FEA016121656FEA0101616590F87C
:100BC000D31D4FEA0161A1656FEA0101E16590F86B
:100BD000D41D4FEA016121666FEA0101616690F858
:100BE000D51D4FEA0161A1666FEA0101E16690F847
:100BF000D61D4FEA016121676FEA0101616790F834
:100C0000D71D4FEA0161A1676FEA0101E16790F822
:100C1000D81D4FEA0161C4F880106FEA0101C4F8E1
:100C2000841090F8D91D4FEA0161C4F888106FEA6A
:100C30000101C4F88C1090F8DA1D4FEA0161C4F884
:100C400090106FEA0101C4F8941090F8DB1D4FEA90
:100C50000161C4F898106FEA0101C4F89C1090F883
:100C6000DC1D4FEA0161C4F8A0106FEA0101C4F86D
:100C7000A41090F8DD1D4FEA0161C4F8A8106FEAD6
:100C80000101C4F8AC1090F8DE1D4FEA0161C4F810
:100C9000B0106FEA0101C4F8B41090F8DF1D4FEAFC
:100CA0000161C4F8B8106FEA0101C4F8BC1090F8F3
:100CB000E01D4FEA0161C4F8C0106FEA0101C4F8F9
:100CC000C41090F8E11D4FEA0161C4F8C8106FEA42
:100CD0000101C4F8CC1090F8E21D4FEA0161C4F89C
:100CE000D0106FEA0101C4F8D41090F8E31D4FEA68
:100CF0000161C4F8D8106FEA0101C4F8DC1004F5F2
:100D0000807490F80F1D4FEA0161A1616FEA010143
:100D1000E16190F8171D4FEA016121624FEA5162CB
:100D200080F863296FEA0101616290F8071D4FEABC
:100D30000161A1636FEA0101E16390F8F01D4FEAE0
:100D4000016121646FEA0101616490F8F11D4FEACD
:100D50000161A1646FEA0101E16490F8F21D4FEABC
:100D6000016121656FEA0101616590F8F31D4FEAA9
:100D70000161A1656FEA0101E16590F8F41D4FEA98
:100D8000016121666FEA0101616690F8F51D4FEA85
:100D90000161A1666FEA0101E16690F8F61D4FEA74
:100DA000016121676FEA0101616790F8F71D4FEA61
:100DB0000161A1676FEA0101E16790F8F81D4FEA50
:100DC0000161C4F880106FEA0101C4F8841090F842
:100DD000F91D4FEA0161C4F888106FEA0101C4F8F7
:100DE0008C1090F8FA1D4FEA0161C4F890106FEA78
:100DF0000101C4F8941090F8FB1D4FEA0161C4F89A
:100E000098106FEA0101C4F89C1090F8FC1D4FEA9D
:100E10000161C4F8A0106FEA0101C4F8A41090F8B1
:100E2000FD1D4FEA0161C4F8A8106FEA0101C4F882
:100E3000AC1090F8FE1D4FEA0161C4F8B0106FEAE3
:100E40000101C4F8B41090F8FF1D4FEA0161C4F825
:100E5000B8106FEA0101C4F8BC1090F8001E4FEA08
:100E60000161C4F8C0106FEA0101C4F8C41090F821
:100E7000011E4FEA0161C4F8C8106FEA0101C4F80D
:100E8000CC1090F8021E4FEA0161C4F8D0106FEA4E
:100E90000101C4F8D41090F8031E4FEA0161C4F8B0
:100EA000D8106FEA0101C4F8DC1004F5807490F8E2
:100EB000101D4FEA0161A1616FEA0101E16190F843
:100EC000181D4FEA016121624FEA516280F8632ADE
:100ED0006FEA0101616290F8081D4FEA0161A163A8
:100EE0006FEA0101E16390F81A1D4FEA0121A0F8B1
:100EF000FA1A90F8101E4FEA016121646FEA0101AD
:100F0000616490F8111E4FEA0161A1646FEA01016A
:100F1000E16490F8121E4FEA016121656FEA010158
:100F2000616590F8131E4FEA0161A1656FEA010146
:100F3000E16590F8141E4FEA016121666FEA010134
:100F4000616690F8151E4FEA0161A1666FEA010122
:100F5000E16690F8161E4FEA016121676FEA010110
:100F6000616790F8171E4FEA0161A1676FEA0101FE
:100F7000E16790F8181E4FEA0161C4F880106FEA2B
:100F80000101C4F8841090F8191E4FEA0161C4F8F9
:100F900088106FEA0101C4F88C1090F81A1E4FEA0D
:100FA0000161C4F890106FEA0101C4F8941090F840
:100FB0001B1E4FEA0161C4F898106FEA0101C4F8E2
:100FC0009C1090F81C1E4FEA0161C4F8A0106FEA53
:100FD0000101C4F8A41090F81D1E4FEA0161C4F885
:100FE000A8106FEA0101C4F8AC1090F81E1E4FEA79
:100FF0000161C4F8B0106FEA0101C4F8B41090F8B0
:101000001F1E4FEA0161C4F8B8106FEA0101C4F86D
:10101000BC1090F8201E4FEA0161C4F8C0106FEABE
:101020000101C4F8C41090F8211E4FEA0161C4F810
:10103000C8106FEA0101C4F8CC1090F8221E4FEAE4
:101040000161C4F8D0106FEA0101C4F8D41090F81F
:10105000231E4FEA0161C4F8D8106FEA0101C4F8F9
:10106000DC1004F5807490F8111D4FEA0161A16154
:101070006FEA0101E16190F8191D4FEA01612162F7
:101080004FEA516280F8632B6FEA0101616290F8C8
:10109000091D4FEA0161A1636FEA0101E16390F864
:1010A0001B1D4FEA0121A0F8FA1B90F8301E4FEAF1
:1010B000016121646FEA0101616490F8311E4FEA19
:1010C0000161A1646FEA0101E16490F8321E4FEA08
:1010D000016121656FEA0101616590F8331E4FEAF5
:1010E0000161A1656FEA0101E16590F8341E4FEAE4
:1010F000016121666FEA0101616690F8351E4FEAD1
:101100000161A1666FEA0101E16690F8361E4FEABF
:10111000016121676FEA0101616790F8371E4FEAAC
:101120000161A1676FEA0101E16790F8381E4FEA9B
:101130000161C4F880106FEA0101C4F8841090F8CE
:10114000391E4FEA0161C4F888106FEA0101C4F842
:101150008C1090F83A1E4FEA0161C4F890106FEAC3
:101160000101C4F8941090F83B1E4FEA0161C4F8E5
:1011700098106FEA0101C4F89C1090F83C1E4FEAE9
:101180000161C4F8A0106FEA0101C4F8A41090F83E
:101190003D1E4FEA0161C4F8A8106FEA0101C4F8CE
:1011A000AC1090F83E1E4FEA0161C4F8B0106FEA2F
:1011B0000101C4F8B41090F83F1E4FEA0161C4F871
:1011C000B8106FEA0101C4F8BC1090F8401E4FEA55
:1011D0000161C4F8C0106FEA0101C4F8C41090F8AE
:1011E000411E4FEA0161C4F8C8106FEA0101C4F85A
:1011F000CC1090F8421E4FEA0161C4F8D0106FEA9B
:101200000101C4F8D41090F8431E4FEA0161C4F8FC
:10121000D8106FEA0101C4F8DC104FF0005041F221
:101220000004C2F2000447F20009C1F2000948F2CA
:101230004007C1F2000702F01AFC4FF0005041F2E3
:101240000004C2F2000447F20009C1F2000948F2AA
:10125000A007C1F2000702F0A8FC4FF0005041F2D5
:101260000001C2F2000147F20007C1F2000703F0DB
:101270003DFD4FF0005000F5807041F20014C2F2C5
:10128000000447F20019C1F2000948F24017C1F208
:10129000000702F0ECFB4FF0005000F5807041F2C7
:1012A0000014C2F2000447F20019C1F2000948F22A
:1012B000A017C1F2000702F078FC4FF0005000F5D3
:1012C000807041F20011C2F2000147F20017C1F232
:1012D000000703F00BFD4FF0005000F5007041F2E5
:1012E0000024C2F2000447F20029C1F2000948F2CA
:1012F0004027C1F2000702F0BAFB4FF0005000F5A2
:10130000007041F20024C2F2000447F20029C1F249
:10131000000948F2A027C1F2000702F046FC4FF096
:10132000005000F5007041F20021C2F2000147F2C6
:101330000027C1F2000703F0D9FC4FF0005000F580
:10134000407041F20034C2F2000447F20039C1F2A9
:10135000000948F24037C1F2000702F088FB4FF065
:10136000005000F5407041F20034C2F2000447F230
:101370000039C1F2000948F2A037C1F2000702F0BB
:1013800014FC4FF0005000F5407041F20031C2F201
:10139000000147F20037C1F2000703F0A7FC4FF04D
:1013A000005000F5806041F20044C2F2000447F2B0
:1013B0000049C1F2000940F20007C4F2010702F03F
:1013C00016FB4FF0005000F5806041F20044C2F27D
:1013D000000447F20049C1F2000948F24047C1F257
:1013E000000702F044FB4FF0005000F5806041F22E
:1013F0000044C2F2000447F20049C1F2000948F279
:10140000A047C1F2000702F0D0FB4FF0005000F5FA
:10141000806041F20041C2F2000147F20047C1F290
:10142000000703F063FC4FF0005000F5A06041F2AC
:101430000054C2F2000447F20059C1F2000944F21C
:101440000007C4F2010702F0D2FA4FF0005000F595
:10145000A06041F20054C2F2000447F20059C1F208
:10146000000948F24057C1F2000702F000FB4FF0BC
:10147000005000F5A06041F20054C2F2000447F2AF
:101480000059C1F2000948F2A057C1F2000702F06A
:101490008CFB4FF0005000F5A06041F20051C2F209
:1014A000000147F20057C1F2000703F01FFC4FF0A4
:1014B000005000F5C06041F20064C2F2000447F23F
:1014C0000069C1F2000940F60007C4F2000702F00B
:1014D000E0F94FF0005000F5C06041F20064C2F244
:1014E000000447F20069C1F2000948F24067C1F206
:1014F000000702F0BCFA4FF0005000F5C06041F266
:101500000064C2F2000447F20069C1F2000948F227
:10151000A067C1F2000702F048FB4FF0005000F551
:10152000C06041F20061C2F2000147F20067C1F2FF
:10153000000703F0DBFB4FF0005000F5E06041F2E4
:101540000074C2F2000447F20079C1F2000940F2CF
:101550000047C4F2000702F09CF94FF0005000F57C
:10156000E06041F20074C2F2000447F20079C1F277
:10157000000948F24077C1F2000702F078FA4FF014
:10158000005000F5E06041F20074C2F2000447F23E
:101590000079C1F2000948F2A077C1F2000702F019
:1015A00004FB4FF0005000F5E06041F20071C2F220
:1015B000000147F20077C1F2000703F097FB4FF0FC
:1015C000005090F8B21000293CD101F1010180F8DF
:1015D000B21043F20043C4F2010341F20004C4F22A
:1015E00002044FF00001C0F21001A16140F2B80105
:1015F000197300BF00BF00BF00BF198911F00201BD
:10160000FBD0198911F08001FBD100BF00BF00BFE2
:1016100000BF00BF00BF00BF00BF00BF00BF40F25F
:101620001001A161998940F60042C4F2000240F223
:101630008501C0F20001116040F20101C0F2000119
:101640005161FBE143F20043C4F2010341F20004A3
:10165000C4F20204218A11F0080140F0EF814FF03A
:10166000000180F8B21040F60042C4F2000240F2DD
:101670000001C0F20001116000BF00BF00BF00BF49
:1016800000BF00BF00BF00BF00BF00BF4FF00001A0
:10169000C0F21001A16140F20001197300BF00BF48
:1016A00000BF00BF198911F00201FBD0198911F0A8
:1016B0008001FBD11E7B06F00F064FEA062690F84C
:1016C000F81E41F0010180F8F81E40F20001197384
:1016D00000BF00BF00BF00BF198911F00201FBD09D
:1016E000198911F08001FBD1197B01F0FF0146EA55
:1016F00001064EF20047C2F200073E80A0F8A86043
:1017000040F20001197300BF00BF00BF00BF19897C
:1017100011F00201FBD0198911F08001FBD11E7B71
:1017200006F00F064FEA062640F20001197300BFCB
:1017300000BF00BF00BF198911F00201FBD0198959
:1017400011F08001FBD1197B01F0FF0146EA01068F
:101750004EF20057C2F200073E80A0F8AA6040F2A5
:101760000001197300BF00BF00BF00BF198911F04D
:101770000201FBD0198911F08001FBD11E7B06F01C
:101780000F064FEA062640F20001197300BF00BFA2
:1017900000BF00BF198911F00201FBD0198911F0B7
:1017A0008001FBD1197B01F0FF0146EA01064EF2F0
:1017B0000067C2F200073E80A0F8AC6040F2000172
:1017C000197300BF00BF00BF00BF198911F00201EB
:1017D000FBD0198911F08001FBD11E7B06F00F06AA
:1017E0004FEA062640F20001197300BF00BF00BF98
:1017F00000BF198911F00201FBD0198911F0800195
:10180000FBD1197B01F0FF0146EA01064EF2007799
:10181000C2F200073E80A0F8AE6040F200011973EA
:1018200000BF00BF00BF00BF198911F00201FBD04B
:10183000198911F08001FBD11E7B06F00F064FEADB
:10184000062640F20001197300BF00BF00BF00BFB1
:10185000198911F00201FBD0198911F08001FBD127
:10186000197B01F0FF0146EA01064EF20007C2F2C1
:1018700000073E80A0F8A06040F20001197300BF8D
:1018800000BF00BF00BF198911F00201FBD0198908
:1018900011F08001FBD11E7B06F00F064FEA0626F1
:1018A00040F20001197300BF00BF00BF00BF1989DB
:1018B00011F00201FBD0198911F08001FBD1197BD5
:1018C00001F0FF0146EA01064EF20017C2F20007DE
:1018D0003E80A0F8A26040F20001197300BF00BF73
:1018E00000BF00BF198911F00201FBD0198911F066
:1018F0008001FBD11E7B06F00F064FEA062640F260
:101900000001197300BF00BF00BF00BF198911F0AB
:101910000201FBD0198911F08001FBD1197B01F084
:10192000FF0146EA01064EF20027C2F200073E80A0
:10193000A0F8A46040F20001197300BF00BF00BF0F
:1019400000BF198911F00201FBD0198911F0800143
:10195000FBD11E7B06F00F064FEA062640F200017F
:10196000197300BF00BF00BF00BF198911F0020149
:10197000FBD0198911F08001FBD1197B01F0FF0127
:1019800046EA01064EF20037C2F200073E80A0F898
:10199000A66000BF00BF00BF00BF40F21001A16100
:1019A0004FF0005042F24C0AC4F2010A4EF6000B0E
:1019B000C2F2000BBAF80060C18D01EB0B02168079
:1019C00001F1020101F0FF01C1854EF60001C2F2F2
:1019D00000014EF60012C2F2000240F2000631F899
:1019E000025B2E449142FAD14FEAD6144FEA962672
:1019F000B0F8B050818B11F4807111D1AE421DD07E
:101A000007D3A6EB0502082A18D341F4807181831D
:101A100006E0A5EB0602082A10D341F48071818309
:101A2000B5420BD004D204F00704072C06D303E020
:101A300004F00704012C01D2A0F8B060FEF7FFBA51
:101A400046F20000C4F202004FF020034FEA0343C5
:101A50008360036C4FF000504EF6003CC2F2000C65
:101A600013F4002308BF0CF1800C3CF8021BA0F813
:101A700088143CF8021BA0F888153CF8021BA0F85B
:101A800088163CF8021BA0F888173CF8021BA0F847
:101A900088183CF8021BA0F888193CF8021BA0F833
:101AA000881A3CF8021BA0F8881B3CF8021BA0F81F
:101AB0005C103CF8021BA0F860103CF8021BA0F878
:101AC00062103CF8021BA0F8641090F84F1011F05F
:101AD000010140F0BF86B0F85C104FF6FF7C614515
:101AE00054D1B0F888C4BCF1000F4FD1B0F888C50C
:101AF000BCF1000F4AD1B0F888C6BCF1000F45D147
:101B0000B0F888C7BCF1000F40D1B0F888C8BCF16C
:101B1000000F3BD1B0F888C9BCF1000F36D1B0F846
:101B200088CABCF1000F31D1B0F888CBBCF1000FEE
:101B30002CD1B0F860C0BCF1000F27D1B0F862C062
:101B4000BCF1000F22D1B0F864C0BCF1000F1DD170
:101B50004FF0010180F84F104FF00001C0F8041160
:101B600048F20001C2F20001C0F8081101F58852E4
:101B70004FF0000341F8043B9142FBD341F2004295
:101B8000C4F2000240F200011160704790F8201189
:101B900000290BD0A1F1010180F8201141F200428F
:101BA000C4F2000240F20001116011E046F200426E
:101BB000C4F20202916D41F00101916541F20042CF
:101BC000C4F2000240F28501116040F2010151614E
:101BD000B0F85E30B0F85C104FEA112223F00F032A
:101BE00023F4706302F0F00C4FEA0C1C02F00E02BA
:101BF00043EA020343EA0C0340F2FF1201EA020146
:101C000041F20012C2F20002D15203F1020340F687
:101C10000022934228BF0023A0F85E30B0F8601085
:101C20004FEA113303F00F0340F6FF7201EA02019D
:101C30004FEA015147F22802C1F20002082B28BFE7
:101C4000083203F007034FEA0323D15002F10402E4
:101C50006FEA0101D150B0F862104FEAD12303F0CE
:101C60001F0340F2FF7201EA02014FEA415147F2BD
:101C70000002C1F20002082B28BF0832102B28BF37
:101C8000083203F007034FEA0323D15002F10402A4
:101C90006FEA0101D150B0F86630B0F864104FEA35
:101CA000112223F0FF0302F0FF0243EA020340F295
:101CB000F812934206D201F0FF0140F60052C2F240
:101CC0000002D15403F1010340F20022934209D3F0
:101CD0004FF00003B0F81C1DA0F86810B0F81E1DEE
:101CE000A0F85610A0F866302DE9F00F4FF0005024
:101CF000B0F888C44FEA0C4CD0F808145CFB01FC27
:101D00008CFA8CFCC0F8D4C46646D0F86C24D0F8A9
:101D1000D07412F0070104BFFF4387FA87F787FAF0
:101D200087F787FA87F7D0F8141457FB01F787FA7B
:101D300086F6D0F8C81448F2000AC1F2000A48F248
:101D4000200BC1F2000B48F24008C1F200080FF26C
:101D5000560302F01F024FEA82027A44974601F0CE
:101D6000FAB901F054B901F0A3B901F039BA01F0A0
:101D700081BA01F0CCBA01F0BEBC01F009BD01F09E
:101D8000EAB901F044B901F093B901F029BA01F0C0
:101D900071BA01F0BCBA01F0AEBC01F0F9BC01F0BF
:101DA0000EBB01F0D6BBC0F8D064D0F8701411F0AF
:101DB000040108BF664648F2600AC1F2000A48F210
:101DC000800BC1F2000B48F2A008C1F20008D0F865
:101DD0007424D0F8D87412F0070104BFFF4387FAC7
:101DE00087F787FA87F787FA87F7D0F8181457FB31
:101DF00001F787FA86F6D0F8CC140FF2560302F0FA
:101E00001F024FEA82027A44974601F0A4B901F01A
:101E1000FEB801F04DB901F0E3B901F02BBA01F0C1
:101E200076BA01F068BC01F0B3BC01F094B901F0DE
:101E3000EEB801F03DB901F0D3B901F01BBA01F0E1
:101E400066BA01F058BC01F0A3BC01F01DBB01F063
:101E5000E9BB0FF2060201F0E3BC4FF0005000F5C1
:101E60008070B0F888C44FEA0C4CD0F808145CFBC2
:101E700001FC8CFA8CFCC0F8D4C46646D0F86C2403
:101E8000D0F8D07412F0070104BFFF4387FA87F738
:101E900087FA87F787FA87F7D0F8141457FB01F70A
:101EA00087FA86F6D0F8C81448F2001AC1F2000A80
:101EB00048F2201BC1F2000B48F24018C1F20008A2
:101EC0000FF2540302F01F024FEA82027A4497464F
:101ED00001F041B901F09BB801F0EAB801F080B916
:101EE00001F0C8B901F013BA01F005BC01F050BC13
:101EF00001F031B901F08BB801F0DAB801F070B936
:101F000001F0B8B901F003BA01F0F5BB01F040BC33
:101F100001F055BA01F01DBBC0F8D064D0F87014C0
:101F200011F0040108BF664648F2601AC1F2000AC7
:101F300048F2801BC1F2000B48F2A018C1F2000861
:101F4000D0F87424D0F8D87412F0070104BFFF430E
:101F500087FA87F787FA87F787FA87F7D0F8181490
:101F600057FB01F787FA86F6D0F8CC140FF254032A
:101F700002F01F024FEA82027A44974601F0EBB862
:101F800001F045B801F094B801F02AB901F072B936
:101F900001F0BDB901F0AFBB01F0FABB01F0DBB855
:101FA00001F035B801F084B801F01AB901F062B956
:101FB00001F0ADB901F09FBB01F0EABB01F064BADA
:101FC00001F030BB0FF2040201F02ABC4FF00050C8
:101FD00000F50070B0F888C44FEA0C4CD0F8081433
:101FE0005CFB01FC8CFA8CFCC0F8D4C46646D0F8CB
:101FF0006C24D0F8D07412F0070104BFFF4387FAB5
:1020000087F787FA87F787FA87F7D0F8141457FB12
:1020100001F787FA86F6D0F8C81448F2002AC1F210
:10202000000A48F2202BC1F2000B48F24028C1F20E
:1020300000080FF2560302F01F024FEA82027A44B0
:10204000974601F088B800F0E2BF01F031B801F026
:10205000C7B801F00FB901F05AB901F04CBB01F05B
:1020600097BB01F078B800F0D2BF01F021B801F0C1
:10207000B7B801F0FFB801F04AB901F03CBB01F07C
:1020800087BB01F09CB901F064BAC0F8D064D0F805
:10209000701411F0040108BF664648F2602AC1F2CC
:1020A000000A48F2802BC1F2000B48F2A028C1F2CE
:1020B0000008D0F87424D0F8D87412F0070104BFD7
:1020C000FF4387FA87F787FA87F787FA87F7D0F809
:1020D000181457FB01F787FA86F6D0F8CC140FF2E4
:1020E000560302F01F024FEA82027A44974601F03B
:1020F00032B800F08CBF00F0DBBF01F071B801F026
:10210000B9B801F004B901F0F6BA01F041BB01F031
:1021100022B800F07CBF00F0CBBF01F061B801F045
:10212000A9B801F0F4B801F0E6BA01F031BB01F052
:10213000ABB901F077BA0FF2060201F071BB4FF0B4
:10214000005000F54070B0F888C44FEA0C4CD0F84D
:1021500008145CFB01FC8CFA8CFCC0F8D4C4664605
:10216000D0F86C24D0F8D07412F0070104BFFF43FC
:1021700087FA87F787FA87F787FA87F7D0F8141472
:1021800057FB01F787FA86F6D0F8C81448F2003AF0
:10219000C1F2000A48F2203BC1F2000B48F240387D
:1021A000C1F200080FF2540302F01F024FEA82024C
:1021B0007A44974600F0CFBF00F029BF00F078BF07
:1021C00001F00EB801F056B801F0A1B801F093BAD1
:1021D00001F0DEBA00F0BFBF00F019BF00F068BF29
:1021E00000F0FEBF01F046B801F091B801F083BAEB
:1021F00001F0CEBA01F0E3B801F0ABB9C0F8D06499
:10220000D0F8701411F0040108BF664648F2603A35
:10221000C1F2000A48F2803BC1F2000B48F2A0383C
:10222000C1F20008D0F87424D0F8D87412F0070175
:1022300004BFFF4387FA87F787FA87F787FA87F79C
:10224000D0F8181457FB01F787FA86F6D0F8CC14AB
:102250000FF2540302F01F024FEA82027A449746BB
:1022600000F079BF00F0D3BE00F022BF00F0B8BF8D
:1022700001F000B801F04BB801F03DBA01F088BAA6
:1022800000F069BF00F0C3BE00F012BF00F0A8BFAD
:1022900000F0F0BF01F03BB801F02DBA01F078BAC0
:1022A00001F0F2B801F0BEB90FF2040201F0B8BAC1
:1022B0004FF0005000F58060B0F888C44FEA0C4C35
:1022C0000FF2040B00F046BED0F86C24D0F8D074A6
:1022D00012F0070104BFFF4387FA87F787FA87F7F1
:1022E00087FA87F7D0F8141457FB01F787FA86F6B8
:1022F000D0F8C81448F2004AC1F2000A48F2204B54
:10230000C1F2000B48F24048C1F200080FF254033A
:1023100002F01F024FEA82027A44974600F01BBF88
:1023200000F075BE00F0C4BE00F05ABF00F0A2BFBE
:1023300000F0EDBF01F0DFB901F02ABA00F00BBFE9
:1023400000F065BE00F0B4BE00F04ABF00F092BFDE
:1023500000F0DDBF01F0CFB901F01ABA01F02FB8DB
:1023600001F0F7B8C0F8D064D0F8701411F004018F
:1023700008BF664648F2604AC1F2000A48F2804B44
:10238000C1F2000B48F2A048C1F20008D0F8742452
:10239000D0F8D87412F0070104BFFF4387FA87F71B
:1023A00087FA87F787FA87F7D0F8181457FB01F7F1
:1023B00087FA86F6D0F8CC140FF2540302F01F020D
:1023C0004FEA82027A44974600F0C5BE00F01FBE75
:1023D00000F06EBE00F004BF00F04CBF00F097BFED
:1023E00001F089B901F0D4B900F0B5BE00F00FBE1C
:1023F00000F05EBE00F0F4BE00F03CBF00F087BF0E
:1024000001F079B901F0C4B901F03EB801F00AB9A0
:102410000FF2040201F004BA4FF0005000F5A06082
:10242000B0F888C44FEA0C4C0FF2040B00F092BDD8
:10243000D0F86C24D0F8D07412F0070104BFFF4329
:1024400087FA87F787FA87F787FA87F7D0F814149F
:1024500057FB01F787FA86F6D0F8C81448F2005AFD
:10246000C1F2000A48F2205BC1F2000B48F240586A
:10247000C1F200080FF2540302F01F024FEA820279
:102480007A44974600F067BE00F0C1BD00F010BE70
:1024900000F0A6BE00F0EEBE00F039BF01F02BB98F
:1024A00001F076B900F057BE00F0B1BD00F000BEFB
:1024B00000F096BE00F0DEBE00F029BF01F01BB9AF
:1024C00001F066B900F07BBF01F043B8C0F8D064FA
:1024D000D0F8701411F0040108BF664648F2605A43
:1024E000C1F2000A48F2805BC1F2000B48F2A0582A
:1024F000C1F20008D0F87424D0F8D87412F00701A3
:1025000004BFFF4387FA87F787FA87F787FA87F7C9
:10251000D0F8181457FB01F787FA86F6D0F8CC14D8
:102520000FF2540302F01F024FEA82027A449746E8
:1025300000F011BE00F06BBD00F0BABD00F050BE5F
:1025400000F098BE00F0E3BE01F0D5B801F020B96C
:1025500000F001BE00F05BBD00F0AABD00F040BE7F
:1025600000F088BE00F0D3BE01F0C5B801F010B98C
:1025700000F08ABF01F056B80FF2040201F050B922
:102580004FF0005000F5C060B0F888C44FEA0C4C22
:102590000FF2040B00F071BCD0F86C24D0F8D074AA
:1025A00012F0070104BFFF4387FA87F787FA87F71E
:1025B00087FA87F7D0F8141457FB01F787FA86F6E5
:1025C000D0F8C81448F2006AC1F2000A48F2206B41
:1025D000C1F2000B48F24068C1F200080FF2540348
:1025E00002F01F024FEA82027A44974600F0B3BD20
:1025F00000F00DBD00F05CBD00F0F2BD00F03ABE91
:1026000000F085BE01F077B801F0C2B800F0A3BDBC
:1026100000F0FDBC00F04CBD00F0E2BD00F02ABEB1
:1026200000F075BE01F067B801F0B2B800F0C7BEA7
:1026300000F08FBFC0F8D064D0F8701411F004011E
:1026400008BF664648F2606AC1F2000A48F2806B31
:10265000C1F2000B48F2A068C1F20008D0F874245F
:10266000D0F8D87412F0070104BFFF4387FA87F748
:1026700087FA87F787FA87F7D0F8181457FB01F71E
:1026800087FA86F6D0F8CC140FF2540302F01F023A
:102690004FEA82027A44974600F05DBD00F0B7BC75
:1026A00000F006BD00F09CBD00F0E4BD00F02FBEC0
:1026B00001F021B801F06CB800F04DBD00F0A7BCEE
:1026C00000F0F6BC00F08CBD00F0D4BD00F01FBEE1
:1026D00001F011B801F05CB800F0D6BE00F0A2BF66
:1026E0000FF2040201F09CB84FF0005000F5E060DA
:1026F000B0F888C44FEA0C4C0FF2020BBDE3D0F8DF
:102700006C24D0F8D07412F0070104BFFF4387FA9D
:1027100087F787FA87F787FA87F7D0F8141457FBFB
:1027200001F787FA86F6D0F8C81448F2007AC1F2A9
:10273000000A48F2207BC1F2000B48F24078C1F257
:1027400000080FF2560302F01F024FEA82027A4499
:10275000974600F000BD00F05ABC00F0A9BC00F0A4
:102760003FBD00F087BD00F0D2BD00F0C4BF01F056
:102770000FB800F0F0BC00F04ABC00F099BC00F0CB
:102780002FBD00F077BD00F0C2BD00F0B4BF00F077
:10279000FFBF00F014BE00F0DCBEC0F8D064D0F87B
:1027A000701411F0040108BF664648F2607AC1F265
:1027B000000A48F2807BC1F2000B48F2A078C1F217
:1027C0000008D0F87424D0F8D87412F0070104BFC0
:1027D000FF4387FA87F787FA87F787FA87F7D0F8F2
:1027E000181457FB01F787FA86F6D0F8CC140FF2CD
:1027F000560302F01F024FEA82027A44974600F025
:10280000AABC00F004BC00F053BC00F0E9BC00F02E
:1028100031BD00F07CBD00F06EBF00F0B9BF00F02C
:102820009ABC00F0F4BB00F043BC00F0D9BC00F04F
:1028300021BD00F06CBD00F05EBF00F0A9BF00F04C
:1028400023BE00F0EFBE0FF2060200F0E9BFBDE8C4
:10285000F00F70472DE9F00FB0F8621011F400424C
:1028600000F0CC8221F40041012930D14EF6002243
:10287000C2F200024FF0000122F8021B22F8021BF4
:1028800022F8021B22F8021B22F8021B22F8021B6C
:1028900022F8021B22F8021B4FF6FF7122F8021BDE
:1028A0004FF0000122F8021B4FF0000122F8021B3A
:1028B0004FF0000122F8021B46F20042C4F202026D
:1028C000916D41F001019165BDE8F00F704702295B
:1028D00040F0F080D0F808614FF00007B0F888149D
:1028E0000C464FEA142401F0FF0104F0FF0406F83F
:1028F000011B06F8014B0F442744B0F888150C461D
:102900004FEA142401F0FF0104F0FF0406F8011B54
:1029100006F8014B0F442744B0F888160C464FEADE
:10292000142401F0FF0104F0FF0406F8011B06F86F
:10293000014B0F442744B0F888170C464FEA142483
:1029400001F0FF0104F0FF0406F8011B06F8014B3B
:102950000F442744B0F888180C464FEA142401F0BD
:10296000FF0104F0FF0406F8011B06F8014B0F44B9
:102970002744B0F888190C464FEA142401F0FF01EF
:1029800004F0FF0406F8011B06F8014B0F4427442E
:10299000B0F8881A0C464FEA142401F0FF0104F045
:1029A000FF0406F8011B06F8014B0F442744B0F85A
:1029B000881B0C464FEA142401F0FF0104F0FF04C9
:1029C00006F8011B06F8014B0F442744C0F80861C4
:1029D0006FEA070707F1010707F0FF07B0F860107B
:1029E000B94230D14EF60022C2F200024FF000018F
:1029F00022F8021B22F8021B22F8021B22F8021BFB
:102A000022F8021B22F8021B22F8021B22F8021BEA
:102A10004FF6FF7122F8021B4FF0000122F8021B53
:102A20004FF0050122F8021B4FF0000122F8021BB3
:102A300046F20042C4F20202916D41F0010191653B
:102A4000BDE8F00F7047D0F80861A6F11006C0F895
:102A500008614EF60022C2F200024FF0000122F897
:102A6000021B22F8021B22F8021B22F8021B22F88A
:102A7000021B22F8021B22F8021B22F8021B4FF64F
:102A8000FF7122F8021B4FF0000122F8021B4FF0E9
:102A9000070122F8021B4FF0000122F8021B46F248
:102AA0000042C4F20202916D41F001019165BDE85E
:102AB000F00F7047032940F02A81D0F808614FF0E9
:102AC0000007B0F888140C464FEA142401F0FF0107
:102AD00004F0FF0406F8011B06F8014B0F442744DD
:102AE000B0F888150C464FEA142401F0FF0104F0F9
:102AF000FF0406F8011B06F8014B0F442744B0F809
:102B000088160C464FEA142401F0FF0104F0FF047C
:102B100006F8011B06F8014B0F442744B0F888174C
:102B20000C464FEA142401F0FF0104F0FF0406F8FC
:102B3000011B06F8014B0F442744B0F888180C46D7
:102B40004FEA142401F0FF0104F0FF0406F8011B12
:102B500006F8014B0F442744B0F888190C464FEA99
:102B6000142401F0FF0104F0FF0406F8011B06F82D
:102B7000014B0F442744B0F8881A0C464FEA14243E
:102B800001F0FF0104F0FF0406F8011B06F8014BF9
:102B90000F442744B0F8881B0C464FEA142401F078
:102BA000FF0104F0FF0406F8011B06F8014B0F4477
:102BB0002744C0F808616FEA070707F1010707F02B
:102BC000FF07B0F86010B9427FF43DAF72B64FF026
:102BD000005043F60042C4F20202D0F80461002E15
:102BE00034D1D16811F48031FBD140F22311C4F209
:102BF0006751516000BF00BF00BF00BFD16811F432
:102C00008031FBD148F6AB11CCF6EF51516000BFDB
:102C100000BF00BF00BFD16811F48031FBD148F282
:102C20000001C0F200011161116941F480311161AC
:102C300000BF00BF00BF00BFD16811F48031FBD1DD
:102C40004FF00006C0F61006C0F8046148F2000517
:102C5000C2F2000505F5805740F20121C0F20001E3
:102C6000116100BF00BF55F8041B46F8041B00BFEC
:102C700000BF00BF00BFD16811F48031FBD1BD425D
:102C8000F1D3C0F80461116921F00101116162B64C
:102C900048F20005C2F20005C0F8085105F580565B
:102CA0004FF0000145F8041BB542FBD34EF600225D
:102CB000C2F200024FF0000122F8021B22F8021BB0
:102CC00022F8021B22F8021B22F8021B22F8021B28
:102CD00022F8021B22F8021B4FF6FF7122F8021B9A
:102CE0004FF0000122F8021B4FF0060122F8021BF0
:102CF0004FF0000122F8021B46F20042C4F2020229
:102D0000916D41F001019165BDE8F00F7047042914
:102D100071D172B64FF0005043F60042C4F2020285
:102D20004FF6F076C0F6170640F20121C0F200011E
:102D3000116100BF00BFB0F88814B0F888454FEAB1
:102D4000044441EA040146F8041B00BF00BF00BF71
:102D500000BFD16811F48031FBD100BF00BFB0F8D3
:102D60008816B0F888474FEA044441EA040146F85F
:102D7000041B00BF00BF00BF00BFD16811F4803149
:102D8000FBD1116921F001011161116941F000418C
:102D9000116162B64EF60022C2F200024FF000014D
:102DA00022F8021B22F8021B22F8021B22F8021B47
:102DB00022F8021B22F8021B22F8021B22F8021B37
:102DC0004FF6FF7122F8021B4FF0000122F8021BA0
:102DD0004FF0080122F8021B4FF0000122F8021BFD
:102DE00046F20042C4F20202916D41F00101916588
:102DF000BDE8F00F7047BDE8F00F70474EF60022B7
:102E0000C2F20002B0F8881422F8021BB0F888154C
:102E100022F8021BB0F8881622F8021BB0F88817B7
:102E200022F8021BB0F8881822F8021BB0F88819A3
:102E300022F8021BB0F8881A22F8021BB0F8881B8F
:102E400022F8021BB0F85C1022F8021BB0F86010E8
:102E500022F8021BB0F8621022F8021BB0F86410CE
:102E600022F8021B46F20042C4F20202916D41F0C8
:102E700001019165BDE8F00F7047D0F86814002992
:102E800009D1D0F808145CFB01FC8CFA8CFCC0F86A
:102E9000D4C466465DE0012919D1D0F804146FF05E
:102EA000000CD0F8E4544FEA510101F100418D4289
:102EB00038BF4FF0000C0CF1004CD0F808145CFB4C
:102EC00001FC8CFA8CFCC0F8D4C4664641E00629AB
:102ED00001D0022909D1D0F808145CFB01FC8CFA5E
:102EE0008CFCC0F8D4C4664633E003291CD14FF0F3
:102EF00040416FF00009D0F8E4548D4238BF4FF0E4
:102F0000000909F10049D0F808145CFB01FC8CFAB7
:102F10008CF6C0F8D464B0F8E8144FEA815159FB3C
:102F200001F989FA89FC14E0042909D1D0F80814C0
:102F30005CFB01FC8CFA8CFCC0F8D4C4664608E04B
:102F4000D0F808145CFB01FC8CFA8CFCC0F8D4C4EB
:102F50006646DF46D0F86814002909D1D0F8081475
:102F60005CFB01FC8CFA8CFCC0F8D4C466464DE0D6
:102F7000012909D1D0F808145CFB01FC8CFA8CFC07
:102F8000C0F8D4C4664641E0062901D0022909D11F
:102F9000D0F808145CFB01FC8CFA8CFCC0F8D4C49B
:102FA000664633E003291CD14FF040416FF0000921
:102FB000D0F8E4548D4238BF4FF0000909F10049C0
:102FC000D0F808145CFB01FC8CFA8CF6C0F8D464D1
:102FD000B0F8E8144FEA815159FB01F989FA89FCEC
:102FE00014E0042909D1D0F808145CFB01FC8CFA28
:102FF0008CFCC0F8D4C4664608E0D0F808145CFB2A
:1030000001FC8CFA8CFCC0F8D4C46646DF464FEA5B
:10301000910101F5803156FB01F6CAF800604FEAD4
:10302000660258F8045B55FB0622DBF800404FEAC5
:10303000640482FA82F758F8045B55FB064458F89A
:10304000045B55FB074484FA84F54AF8045B82FA72
:1030500082F6DAF8002058F8045B55FB0622DBF80C
:1030600000404FEA640482FA82F758F8045B55FB8B
:10307000064458F8045B55FB074484FA84F54AF883
:10308000045B58F8045B55FB06F482FA82F658F8A4
:10309000045B55FB074484FA84F54BF8045B86FA1D
:1030A00086F686FA86F686FA86F686FA86F69F46CB
:1030B0004FEA910101F5803156FB01F6CAF8006034
:1030C0004FEA660258F8045B55FB0622DBF8004025
:1030D0004FEA640482FA82F758F8045B55FB064411
:1030E00058F8045B55FB074484FA84F54AF8045BFE
:1030F00082FA82F6DAF8002058F8045B55FB0622C3
:10310000DBF800404FEA640482FA82F758F8045B67
:1031100055FB064458F8045B55FB074484FA84F5D4
:103120004AF8045B58F8045B55FB06F482FA82F611
:1031300058F8045B55FB074484FA84F54BF8045BAC
:1031400086FA86F686FA86F686FA86F686FA86F68F
:1031500086FA86F69F464FEAA606CAF800604FEA4E
:10316000660258F8045B55FB0622DBF800404FEA84
:10317000640482FA82F758F8045B55FB064458F859
:10318000045B55FB074484FA84F54AF8045B82FA31
:1031900082F6DAF8002058F8045B55FB0622DBF8CB
:1031A00000404FEA640482FA82F758F8045B55FB4A
:1031B000064458F8045B55FB074484FA84F54AF842
:1031C000045B58F8045B55FB06F482FA82F658F863
:1031D000045B55FB074484FA84F54BF8045B9F4677
:1031E0004FEAA606B146CAF800604FEA660258F8F0
:1031F000045B55FB0622DBF800404FEA640482FAC8
:1032000082F758F8045B55FB064458F8045B55FBFD
:10321000074484FA84F54AF8045B82FA82F6DAF805
:10322000002058F8045B55FB0622DBF800404FEA0B
:10323000640482FA82F758F8045B55FB064458F898
:10324000045B55FB074484FA84F54AF8045B58F89C
:10325000045B55FB06F482FA82F658F8045B55FBD2
:10326000074484FA84F54BF8045B6FEA060689FA92
:1032700086F69F464FEA910101F1806156FB01F607
:103280004FEAE606CAF800604FEA660258F8045BA7
:1032900055FB0622DBF800404FEA640482FA82F70D
:1032A00058F8045B55FB064458F8045B55FB07448B
:1032B00084FA84F54AF8045B82FA82F6DAF8002090
:1032C00058F8045B55FB0622DBF800404FEA640423
:1032D00082FA82F758F8045B55FB064458F8045B01
:1032E00055FB074484FA84F54AF8045B58F8045BFC
:1032F00055FB06F482FA82F658F8045B55FB074446
:1033000084FA84F54BF8045B86FA86F69F46B1464C
:103310004FEA910101F5803156FB01F6CAF80060D1
:103320004FEA660258F8045B55FB0622DBF80040C2
:103330004FEA640482FA82F758F8045B55FB0644AE
:1033400058F8045B55FB074484FA84F54AF8045B9B
:1033500082FA82F6DAF8002058F8045B55FB062260
:10336000DBF800404FEA640482FA82F758F8045B05
:1033700055FB064458F8045B55FB074484FA84F572
:103380004AF8045B58F8045B55FB06F482FA82F6AF
:1033900058F8045B55FB074484FA84F54BF8045B4A
:1033A00086FA86F686FA86F686FA86F686FA86F62D
:1033B0004FEA69096FEA060689FA86F69F46B14622
:1033C0004FEA910101F5803156FB01F6CAF8006021
:1033D0004FEA660258F8045B55FB0622DBF8004012
:1033E0004FEA640482FA82F758F8045B55FB0644FE
:1033F00058F8045B55FB074484FA84F54AF8045BEB
:1034000082FA82F6DAF8002058F8045B55FB0622AF
:10341000DBF800404FEA640482FA82F758F8045B54
:1034200055FB064458F8045B55FB074484FA84F5C1
:103430004AF8045B58F8045B55FB06F482FA82F6FE
:1034400058F8045B55FB074484FA84F54BF8045B99
:1034500086FA86F686FA86F686FA86F686FA86F67C
:10346000B0F8DC244FEAC25212F000470CBFD2433E
:10347000F64322F0004256FB02F686FA86F64FEA41
:10348000690989FA86F69F46B1464FEA910101F52E
:10349000803156FB01F6CAF800604FEA660258F820
:1034A000045B55FB0622DBF800404FEA640482FA15
:1034B00082F758F8045B55FB064458F8045B55FB4B
:1034C000074484FA84F54AF8045B82FA82F6DAF853
:1034D000002058F8045B55FB0622DBF800404FEA59
:1034E000640482FA82F758F8045B55FB064458F8E6
:1034F000045B55FB074484FA84F54AF8045B58F8EA
:10350000045B55FB06F482FA82F658F8045B55FB1F
:10351000074484FA84F54BF8045B86FA86F686FA4B
:1035200086F686FA86F686FA86F6B0F8E0244FEA42
:10353000C25212F000470CBFD243F64322F00042C1
:1035400056FB02F686FA86F64FEA690989FA86F68C
:103550009F46B1464FEA910101F5803156FB01F6D5
:10356000CAF800604FEA660258F8045B55FB062271
:10357000DBF800404FEA640482FA82F758F8045BF3
:1035800055FB064458F8045B55FB074484FA84F560
:103590004AF8045B82FA82F6DAF8002058F8045BF5
:1035A00055FB0622DBF800404FEA640482FA82F7FA
:1035B00058F8045B55FB064458F8045B55FB074478
:1035C00084FA84F54AF8045B58F8045B55FB06F46A
:1035D00082FA82F658F8045B55FB074484FA84F5B6
:1035E0004BF8045B86FA86F686FA86F686FA86F645
:1035F00086FA86F686FA86F686FA86F6B0F8DC242F
:103600004FEAC25212F000470CBFD243F64322F0F9
:10361000004256FB02F686FA86F64FEA690989FAF5
:1036200086F69F46B1464FEA910101F5803156FB7F
:1036300001F6CAF800604FEA660258F8045B55FBD1
:103640000622DBF800404FEA640482FA82F758F859
:10365000045B55FB064458F8045B55FB074484FAA9
:1036600084F54AF8045B82FA82F6DAF8002058F80A
:10367000045B55FB0622DBF800404FEA640482FA43
:1036800082F758F8045B55FB064458F8045B55FB79
:10369000074484FA84F54AF8045B58F8045B55FB48
:1036A00006F482FA82F658F8045B55FB074484FA64
:1036B00084F54BF8045B86FA86F686FA86F686FA77
:1036C00086F686FA86F686FA86F686FA86F6B0F8E2
:1036D000E0244FEAC25212F000470CBFD243F64337
:1036E00022F0004256FB02F686FA86F64FEA690996
:1036F00089FA86F69F464FEA910101F1806156FBF7
:1037000001F6CAF800604FEA660258F8045B55FB00
:103710000622DBF800404FEA640482FA82F758F888
:10372000045B55FB064458F8045B55FB074484FAD8
:1037300084F54AF8045B82FA82F6DAF8002058F839
:10374000045B55FB0622DBF800404FEA640482FA72
:1037500082F758F8045B55FB064458F8045B55FBA8
:10376000074484FA84F54AF8045B58F8045B55FB77
:1037700006F482FA82F658F8045B55FB074484FA93
:1037800084F54BF8045B86FA86F686FA86F69F4641
:103790004FEA910101F1806156FB01F6CAF8006021
:1037A0004FEA660258F8045B55FB0622DBF800403E
:1037B0004FEA640482FA82F758F8045B55FB06442A
:1037C00058F8045B55FB074484FA84F54AF8045B17
:1037D00082FA82F6DAF8002058F8045B55FB0622DC
:1037E000DBF800404FEA640482FA82F758F8045B81
:1037F00055FB064458F8045B55FB074484FA84F5EE
:103800004AF8045B58F8045B55FB06F4164658F872
:10381000045B55FB074484FA84F54BF8045B9F4630
:10382000C0F8D864D0F8781411F0010118BFF6433D
:10383000D0F8D0C4D0F8301411F0004904D156FBB0
:1038400001F686FA86F605E06FEA01015CFB01FCF1
:103850008CFA8CFC86FA8CFCD0F8D434D0F82C147A
:103860006FEA010929F000495CFB09FC8CFA8CFC29
:1038700053FB01F383FA83F383FA8CFCD0F85C14D6
:103880005CFB01FC8CFA8CFC8CFA8CFCC0F864C4E8
:103890009746B4F80811002905D140F28401C0F21E
:1038A00000013960A2E0012973D140F26E31B4F811
:1038B0000261A1F580713144B4F8002190F86334BD
:1038C0001A44403A38BF0022802A28BF7F226FEA7C
:1038D000020240F27F0302EA03024FEAC2121144DD
:1038E000B0F8FAA440F22E0B4FEA0A4A0AF1004A55
:1038F0004FEA6A0A4FEA8B5B5AFB0BFA8AFA8AFA9A
:10390000B4F8AA814FEA880809EB080BDBF80080BD
:10391000B4F858B108F100484FEA68084FEA8B5BE9
:1039200058FB0BF888FA88F888FA8AFAB4F8AC8160
:103930004FEA880809EB080BDBF80080B4F8AEB159
:1039400008F100484FEA68084FEA8B5B58FB0BF818
:1039500088FA88F888FA8AFA1AF0004B0DD14FEAF3
:103960009A4AB1EB0A0138BF40F26E2140F26E2A4A
:10397000514538BF40F26E2104E06FEA0A0A4FEA6F
:10398000DA4A5144F96240F28501C0F2000139601F
:103990002CE0062901D0022905D140F28401C0F2B1
:1039A0000001396022E0032913D140F26E21B4F8FE
:1039B00032216FEA020240F2FF1302EA03024FEAE9
:1039C00042121144F96240F28501C0F200013960EF
:1039D0000CE0042905D140F28401C0F200013960F5
:1039E00004E040F28401C0F2000139607047B4F88D
:1039F0000811002905D140F28401C0F200013960AC
:103A000034E0012905D140F28401C0F2000139609F
:103A10002CE0062901D0022905D140F28401C0F230
:103A20000001396022E0032913D140F26E21B4F87D
:103A300032216FEA020240F2FF1302EA03024FEA68
:103A400042121144F96240F28501C0F2000139606E
:103A50000CE0042905D140F28401C0F20001396074
:103A600004E040F28401C0F2000139607047B4F80C
:103A70005C314FEAC313B4F8C4A14FEA8A0A09EBD8
:103A80000A0BDBF800A0B4F866B1BBF1000F1CD044
:103A90000AF1004A4FEA8B5B5AFB0BFA8AFA8AFA60
:103AA0001AF0004B08D14FEA1A4A534413F4803AF3
:103AB0000BD04FF6FF7308E06FEA0A0A4FEA1A4A82
:103AC000B3EB0A0301D24FF00003B4F8C6A14FEAEA
:103AD0008A0A09EB0A0BDBF800A0B4F88EB1BBF13F
:103AE000000F1CD00AF1004A4FEA8B5B5AFB0BFA1D
:103AF0008AFA8AFA1AF0004B08D14FEA1A4A53445C
:103B000013F4803A0BD04FF6FF7308E06FEA0A0A0D
:103B10004FEA1A4AB3EB0A0301D24FF000031946E9
:103B2000B4F85E314FEAC313B4F8CAA14FEA8A0A67
:103B300009EB0A0BDBF800A0B4F8CCB1BBF1000F25
:103B40001CD00AF1004A4FEA8B5B5AFB0BFA8AFA47
:103B50008AFA1AF0004B08D14FEA1A4A534413F478
:103B6000803A0BD04FF6FF7308E06FEA0A0A4FEA7B
:103B70001A4AB3EB0A0301D24FF00003B4F85A21FA
:103B8000B4F86091B4F86261B4F864810D4605FB45
:103B900005F1C0F8C8144FEA11413D462DE9005027
:103BA00000F0A1F8BDE800507047B4F86C314FEA5E
:103BB000C313B4F878A14FEA8A0A09EB0A0BDBF8C1
:103BC00000A0B4F876B1BBF1000F1CD00AF1004A96
:103BD0004FEA8B5B5AFB0BFA8AFA8AFA1AF0004B0F
:103BE00008D14FEA1A4A534413F4803A0BD04FF6E7
:103BF000FF7308E06FEA0A0A4FEA1A4AB3EB0A03B6
:103C000001D24FF00003B4F8D2A14FEA8A0A09EBBF
:103C10000A0BDBF800A0B4F890B1BBF1000F1CD088
:103C20000AF1004A4FEA8B5B5AFB0BFA8AFA8AFACE
:103C30001AF0004B08D14FEA1A4A534413F4803A61
:103C40000BD04FF6FF7308E06FEA0A0A4FEA1A4AF0
:103C5000B3EB0A0301D24FF000031946B4F86E31FA
:103C60004FEAC313B4F8D6A14FEA8A0A09EB0A0B4C
:103C7000DBF800A0B4F8D8B1BBF1000F1CD00AF1FA
:103C8000004A4FEA8B5B5AFB0BFA8AFA8AFA1AF05F
:103C9000004B08D14FEA1A4A534413F4803A0BD030
:103CA0004FF6FF7308E06FEA0A0A4FEA1A4AB3EBCD
:103CB0000A0301D24FF00003B4F86A21B4F87091FE
:103CC000B4F87261B4F874810D4605FB05F1C0F8D3
:103CD000CC144FEA11413D462DE9005000F003F8A5
:103CE000BDE80050704702F01F024FEA82027A449A
:103CF000974600F0E6B900F020B800F0A6B800F052
:103D000057BA00F0C6BA00F03BBB00F0A5BB00F00C
:103D100014BC00F089BC00F0F4BC00F05EBD00F003
:103D2000C8BD00F033BE00F09DBE00F007BF00F03C
:103D300070BF00F0F6B800F05CB940F2004740F206
:103D4000003B0BFB01FB4FEA0747A7EB0B0745F8CE
:103D5000047B40F2000740F2000B45F8047B47F675
:103D6000002744F2002B0BFB01FB4FEA0747A7EBB0
:103D70000B0745F8047B40F200274FEA49094F44FE
:103D800040F2001B0BFB01FB4FEA07475F4445F87D
:103D9000047B40F2000740F2000B45F8047B47F635
:103DA000007744F2001B0BFB01FB4FEA0747A7EB30
:103DB0000B0745F8047B4FF600574FEA0818A7EBAE
:103DC000080740F2001B0BFB01FB4FEA0747A7EB7C
:103DD0000B0745F8047B4CF200174CF200143444F6
:103DE000A4EB07046FEA03034FF6FF7203EA020332
:103DF00004FB03F44FEA144427444CF2003B4FF217
:103E00000034A4EB0B0404FB03F44FEA1444A34472
:103E1000BB4515D009D3ABEB070B0BFB01FB4FEAFE
:103E200007475F4445F8047B7047A7EB0B0B0BFB80
:103E300001FB4FEA0747A7EB0B0745F8047B7047E8
:103E40004FEA074745F8047B704740F2CD1740F230
:103E5000930B0BFB01FB4FEA0747A7EB0B0745F85A
:103E6000047B40F2000740F2000B45F8047B47F664
:103E70003E5745F2434B0BFB01FB4FEA0747A7EBCD
:103E80000B0745F8047B40F22E274FEA49094F44BF
:103E900040F2071B0BFB01FB4FEA07475F4445F865
:103EA000047B40F2000740F2000B45F8047B47F624
:103EB0001F7744F6A26B0BFB01FB4FEA0747A7EB0A
:103EC0000B0745F8047B4FF6D2574FEA0818A7EBCB
:103ED000080740F2071B0BFB01FB4FEA0747A7EB64
:103EE0000B0745F8047B4CF2CF074CF2E004344456
:103EF000A4EB07046FEA03034FF6FF7203EA020321
:103F000004FB03F44FEA144427444CF2811B4FF2A4
:103F10000044A4EB0B0404FB03F44FEA1444A34451
:103F200076E740F2004740F2003B0BFB01FB4FEA13
:103F30000747A7EB0B0745F8047B40F2000740F268
:103F4000000B45F8047B47F6002744F2002B0BFBDF
:103F500001FB4FEA0747A7EB0B0745F8047B40F24C
:103F600000274FEA49094F4440F2001B0BFB01FBBD
:103F70004FEA07475F4445F8047B40F2000740F2F0
:103F8000000B45F8047B47F6007744F2001B0BFB5F
:103F900001FB4FEA0747A7EB0B0745F8047B4FF6F9
:103FA000005740F2001B0BFB01FB4FEA0747A7EB52
:103FB0000B0745F8047B4CF200174CF20014344414
:103FC000A4EB07046FEA03034FF6FF7203EA020350
:103FD00004FB03F44FEA144427444CF2003B4FF235
:103FE0000034A4EB0B0404FB03F44FEA1444A34491
:103FF0000EE740F2CD1740F2930B0BFB01FB4FEAAB
:104000000747A7EB0B0745F8047B40F2000740F297
:10401000000B45F8047B47F63E5745F2434B0BFB3C
:1040200001FB4FEA0747A7EB0B0745F8047B40F27B
:104030002E274FEA49094F4440F2071B0BFB01FBB7
:104040004FEA07475F4445F8047B40F2000740F21F
:10405000000B45F8047B47F61F7744F6A26B0BFB79
:1040600001FB4FEA0747A7EB0B0745F8047B4FF628
:10407000D25740F2071B0BFB01FB4FEA0747A7EBA8
:104080000B0745F8047B4CF2CF074CF2E0043444B4
:10409000A4EB07046FEA03034FF6FF7203EA02037F
:1040A00004FB03F44FEA144427444CF2811B4FF203
:1040B0000044A4EB0B0404FB03F44FEA1444A344B0
:1040C000A6E640F2010740F6FF0B0BFB01FB4FEAAF
:1040D00007475F4445F8047B40F2030741F2BD2BDC
:1040E0000BFB01FB4FEA07475F4445F8047B47F6AB
:1040F000F16745F2712B0BFB01FB4FEA0747A7EB7A
:104100000B0745F8047B40F2020740F6BE4B0BFB61
:1041100001FB4FEA07475F4445F8047B40F2040780
:104120004FEA89094F4441F67C1BABEB090B0BFBB3
:1041300001FB4FEA07475F4445F8047B47F6FC67FD
:1041400044F6FA5B0BFB01FB4FEA0747A7EB0B07B3
:1041500045F8047B40F202074FEA4808474440F61E
:10416000BE4B0BFB01FB4FEA07475F4445F8047B5E
:104170004CF204174CF204144FEA96063444A4EBB4
:1041800007046FEA03034FF6FF7203EA020304FB1E
:1041900003F44FEA144427444DF6C01B4FF6C014F5
:1041A000A4EB0B0404FB03F44FEA1444A3442FE6EE
:1041B00040F2010740F6FF0B0BFB01FB4FEA0747FC
:1041C0005F4445F8047B40F2030741F2BD2B0BFB33
:1041D00001FB4FEA07475F4445F8047B47F6F16768
:1041E00045F2712B0BFB01FB4FEA0747A7EB0B07CF
:1041F00045F8047B40F202074FEA4808474440F67E
:10420000BE4B0BFB01FB4FEA07475F4445F8047BBD
:1042100040F204074F4441F67C1B0BFB01FB4FEAC5
:1042200007475F4445F8047B47F6FC6744F6FA5BB2
:104230000BFB01FB4FEA0747A7EB0B0745F8047B95
:1042400040F20207374440F6BE4B0BFB01FB4FEA3E
:1042500007475F4445F8047B4CF204174CF2041402
:10426000A4EB07046FEA03034FF6FF7203EA0203AD
:1042700004FB03F44FEA144427444DF6C01B4FF6E9
:10428000C014A4EB0B0404FB03F44FEA1444A3444E
:10429000BEE543F6FF7741F62B1B0BFB01FB4FEA14
:1042A0000747A7EB0B0745F8047B48F2010746F2E6
:1042B000444B0BFB01FB4FEA07475F4445F8047B87
:1042C00046F6FC7743F6FA1B0BFB01FB4FEA074768
:1042D000A7EB0B0745F8047B42F2000744F2794B49
:1042E0000BFB01FB4FEA07475F4445F8047B4FF2A5
:1042F00000074FEA8919A7EB090743F2BF7B0BFBC5
:1043000001FB4FEA0747A7EB0B0745F8047B47F68D
:10431000FE774FEA8808A7EB080744F6EC4B0BFB47
:1043200001FB4FEA0747A7EB0B0745F8047B42F276
:10433000000744F2794B0BFB01FB4FEA07475F4450
:1043400045F8047B4CF200074CF210043444A4EB13
:1043500007046FEA03034FF6FF7203EA020304FB4C
:1043600003F44FEA144427444CF2D32B4FF2C024F9
:10437000A4EB0B0404FB03F44FEA1444A34447E505
:1043800040F2004740F2003B0BFB01FB4FEA0747BE
:10439000A7EB0B0745F8047B40F2000740F2000B47
:1043A00045F8047B47F6002744F2002B0BFB01FB8A
:1043B0004FEA0747A7EB0B0745F8047B40F20027BD
:1043C00040F2001B0BFB01FB4FEA07475F4445F837
:1043D000047B40F2000740F2000B45F8047B47F6EF
:1043E00000774F4444F2001B0BFB01FB4FEA0747E9
:1043F000A7EB0B0745F8047B4FF600574FEA46063C
:1044000037444FEA0818A7EB080740F2001B0BFBE4
:1044100001FB4FEA0747A7EB0B0745F8047B4CF27B
:1044200000174CF20014A4EB07046FEA03034FF6E5
:10443000FF7203EA020304FB03F44FEA1444274427
:104440004CF2003B4FF20034A4EB0B0404FB03F4EA
:104450004FEA1444A344DBE440F2CD1740F2930B3F
:104460000BFB01FB4FEA0747A7EB0B0745F8047B63
:1044700040F2000740F2000B45F8047B47F63E5738
:1044800045F29E3B0BFB01FB4FEA0747A7EB0B07EF
:1044900045F8047B40F22E274FEA09194F4440F2B9
:1044A000071B0BFB01FB4FEA07475F4445F8047B02
:1044B00040F2000740F2000B45F8047B47F61F77F7
:1044C0004FEA8606A7EB060744F6A26BABEB060B9A
:1044D0000BFB01FB4FEA0747A7EB0B0745F8047BF3
:1044E00040F280074FEA8808474440F6F94BABEBAF
:1044F000080B0BFB01FB4FEA07475F4445F8047BC1
:104500004CF2A4074CF2C404A4EB07046FEA0303C3
:104510004FF6FF7203EA020304FB03F44FEA14446C
:1045200027444CF6C01B4FF6C014A4EB0B0404FB4D
:1045300003F44FEA1444A3446AE440F2CD1740F276
:10454000930B0BFB01FB4FEA0747A7EB0B0745F863
:10455000047B40F2000740F2000B45F8047B47F66D
:104560003E5747F29E3B0BFB01FB4FEA0747A7EB89
:104570000B0745F8047B40F200074AF2000B0BFBE7
:1045800001FB4FEA07475F4445F8047B40F2000710
:104590004FEA49194F4440F6000B0BFB01FB4FEA71
:1045A00007475F4445F8047B47F6FC674FEA061669
:1045B000A7EB060744F6FA5B0BFB01FB4FEA074744
:1045C000A7EB0B0745F8047B47F600774FEA8818FE
:1045D000A7EB080745F2006BABEB060B0BFB01FBEF
:1045E0004FEA0747A7EB0B0745F8047B4BF6CF27AD
:1045F0004CF2E014A4EB07046FEA03034FF6FF72DA
:1046000003EA020304FB03F44FEA144427444AF28A
:10461000810B4FF20044A4EB0B0404FB03F44FEABC
:104620001444A344FFF7F4BB40F2010740F6001B1B
:1046300004B5FFF7EDFBBDE8044040F2030741F28B
:10464000C02B04B5FFF7E4FBBDE8044047F6F16773
:1046500042F6804B04B5FFF7DBFBBDE8044040F2B7
:10466000020740F6C04B04B5FFF7D2FBBDE804409B
:1046700040F2040741F6801B4FEA09194F44ABEBA7
:10468000090B04B5FFF7C4FBBDE8044047F6FC671F
:1046900043F2021B4FEA4606A7EB0607B3444FEA74
:1046A0008808A7EB0807ABEB080B04B5FFF7B0FBD6
:1046B000BDE8044040F2020740F6C04B04B5FFF7E6
:1046C000A7FBBDE804404CF204174CF21414A4EB11
:1046D00007046FEA03034FF6FF7203EA020304FBC9
:1046E00003F44FEA144427444DF6C01B4FF6C014A0
:1046F000A4EB0B0404FB03F44FEA1444A344FFF7B8
:1047000087BB40F2004740F2001B04B5FFF780FB77
:10471000BDE8044040F2000740F2000B04B5FFF78B
:1047200077FBBDE8044047F6002743F6000B04B5CD
:10473000FFF76EFBBDE8044040F2002740F2003B6B
:104740004FEA49094F44CB4404B5FFF761FBBDE88C
:10475000044040F2000740F2000B04B5FFF758FB9D
:10476000BDE8044047F6007743F6006B4FEA860643
:10477000A7EB0607B34404B5FFF74AFBBDE80440C6
:104780004FF600574FF6004B4FEA8818A7EB080783
:10479000ABEB080B04B5FFF73BFBBDE804404CF264
:1047A00000174CF21014A4EB07046FEA03034FF652
:1047B000FF7203EA020304FB03F44FEA14442744A4
:1047C0004CF2003B4FF20034A4EB0B0404FB03F467
:1047D0004FEA1444A344FFF71BBB40F2CD1740F24D
:1047E0003A1B04B5FFF714FBBDE8044040F2000794
:1047F00040F2000B04B5FFF70BFBBDE8044047F6A1
:104800003E5742F6A01B04B5FFF702FBBDE804408B
:1048100040F22E2740F2353B4FEA49094F44CB4442
:1048200004B5FFF7F5FABDE8044040F2000740F296
:10483000000B04B5FFF7ECFABDE8044047F61F771C
:1048400043F27D0B4FEA8606A7EB0607B34404B597
:10485000FFF7DEFABDE804404FF6D2574FF6CB4BD8
:104860004FEA8818A7EB0807ABEB080B04B5FFF776
:10487000CFFABDE804404CF2CF074CF2E004A4EBC1
:1048800007046FEA03034FF6FF7203EA020304FB17
:1048900003F44FEA144427444CF2811B4FF20044C6
:1048A000A4EB0B0404FB03F44FEA1444A344FFF706
:1048B000AFBA40F2010740F6001B04B5FFF7A8FAB3
:1048C000BDE8044040F2030741F2C02B04B5FFF7F6
:1048D0009FFABDE8044047F6F16742F6804B04B505
:1048E000FFF796FABDE8044040F2020740F6C04BDD
:1048F00004B5FFF78DFABDE8044040F2040741F625
:10490000801B04B5FFF784FABDE8044047F6FC6756
:1049100043F2021B4FEA4606A7EB0607B3444FEAF1
:104920008909A7EB0907ABEB090B04B5FFF770FA90
:10493000BDE8044040F2020740F6C04B4FEA880849
:104940004744ABEB080B04B5FFF762FABDE804403F
:104950004CF204174CF21414A4EB07046FEA03039F
:104960004FF6FF7203EA020304FB03F44FEA144418
:1049700027444DF6C01B4FF6C014A4EB0B0404FBF8
:1049800003F44FEA1444A344FFF742BA43F6FF7717
:1049900042F2D46B04B5FFF73BFABDE8044048F29D
:1049A00001074EF2454B04B5FFF732FABDE804406B
:1049B00046F6FC7743F2026B04B5FFF729FABDE82F
:1049C000044042F2000746F2794B04B5FFF720FAA3
:1049D000BDE804404CF200074BF6410B4FEAC90911
:1049E0004F44CB4404B5FFF713FABDE8044047F643
:1049F000FE7743F2123B4FEA0616A7EB0607ABEB36
:104A0000060B04B5FFF704FABDE8044042F20007C4
:104A100046F2794B4FEA88084744ABEB080B04B5E4
:104A2000FFF7F6F9BDE804404CF200074CF2100421
:104A3000A4EB07046FEA03034FF6FF7203EA0203D5
:104A400004FB03F44FEA144427444CF2D32B4FF2F7
:104A5000C024A4EB0B0404FB03F44FEA1444A34466
:104A6000FFF7D6B940F2004740F2001B04B5FFF74C
:104A7000CFF9BDE8044040F2000740F2000B04B556
:104A8000FFF7C6F9BDE8044047F6002743F6000BE0
:104A900004B5FFF7BDF9BDE8044040F2002740F23D
:104AA000003B4FEA49094F44CB4404B5FFF7B0F946
:104AB000BDE8044040F2000740F2000B04B5FFF7E8
:104AC000A7F9BDE8044047F6007743F6006B4FEACC
:104AD0008606A7EB0607B34404B5FFF799F9BDE8CE
:104AE00004404FF600574FF6004B4FEA8818A7EBEB
:104AF0000807ABEB080B04B5FFF78AF9BDE80440E3
:104B00004CF200174CF21014A4EB07046FEA0303F5
:104B10004FF6FF7203EA020304FB03F44FEA144466
:104B200027444CF2003B4FF20034A4EB0B0404FB8F
:104B300003F44FEA1444A344FFF76AB940F2CD17D7
:104B400040F23A1B04B5FFF763F9BDE8044040F2B8
:104B5000000740F2000B04B5FFF75AF9BDE8044026
:104B600047F63E5742F6A01B04B5FFF751F9BDE8E2
:104B7000044040F22E2740F2353B4FEA09194F44DA
:104B8000CB4404B5FFF744F9BDE8044040F2000708
:104B900040F2000B04B5FFF73BF9BDE8044047F6CF
:104BA0001F7743F27D0B4FEA8606A7EB0607B34457
:104BB00004B5FFF72DF9BDE8044040F2800740F648
:104BC000795B4FEA88084744ABEB080B04B5FFF765
:104BD0001FF9BDE804404CF204074CF27414A4EB36
:104BE00007046FEA03034FF6FF7203EA020304FBB4
:104BF00003F44FEA144427444CF6C01B4FF6C0148C
:104C0000A4EB0B0404FB03F44FEA1444A344FFF7A2
:104C1000FFB840F2CD1740F23A1B04B5FFF7F8F8A1
:104C2000BDE8044040F2000740F2000B04B5FFF776
:104C3000EFF8BDE8044047F63E5742F6A01B04B526
:104C4000FFF7E6F8BDE8044040F22E2740F2353B7E
:104C500004B5FFF7DDF8BDE804404CF2000740F66C
:104C6000410B4FEA4919A7EB0907CB4404B5FFF7FD
:104C7000CFF8BDE8044047F6FC6745F2021B4FEA57
:104C80004616A7EB0607ABEB060B04B5FFF7C0F81B
:104C9000BDE8044043F6007742F6001B4FEA0818CF
:104CA0004744ABEB080B04B5FFF7B2F8BDE804408E
:104CB0004CF2CF074CF2E004A4EB07046FEA0303C5
:104CC0004FF6FF7203EA020304FB03F44FEA1444B5
:104CD00027444CF2811B4FF20044A4EB0B0404FB6D
:104CE00003F44FEA1444A344FFF792B83B694FEA38
:104CF0005303C0F85C34B1F80631B1F8B421B1F80F
:104D0000B6B12DE9005000F08BF8BDE80050C0F8B6
:104D10000434B1F80E31B1F8B821B1F8BAB12DE9C7
:104D2000005000F07DF8BDE800504FEA5303C0F892
:104D30000834B1F88631B1F8CE21B1F8D0B12DE9FF
:104D4000005000F06DF8BDE800504FEA5303C0F882
:104D50001434B1F88831B1F8DA21B1F8DCB12DE9B9
:104D6000005000F05DF8BDE800504FEA5303C0F872
:104D70001834B1F88A31B1F8EE21B1F8F0B12DE96B
:104D8000005000F04DF8BDE800504FEA5303C0F862
:104D90002C34B1F86831B1F8F221B1F8F4B12DE951
:104DA000005000F03DF8BDE80050C0F83034B1F8D4
:104DB000A831B1F8F621B1F8F8B10BFB03FB4FEACB
:104DC0005B2B2DE9005000F02BF8BDE800504FEAB6
:104DD0005303C0F83434B1F87A31C0F87034B1F804
:104DE0005A31C0F86C34B1F86A31C0F87434B1F893
:104DF0006431C0F8DC34B1F87431C0F8E034B1F893
:104E00008431C0F87834B1F80831C0F86834B1F8AA
:104E1000AC31A0F88C34B1F80A31A0F8E83470470E
:104E20004FEAC3534FEA820257F802A0BBF1000FCA
:104E300016D00AF1004A4FEA8B5B5AFB0BFA8AFA4A
:104E40008AFA1AF0004B05D113EB0A0328BF6FF062
:104E5000000370476FEA0A0AB3EB0A0338BF002366
:104E6000704772B646F20040C4F202004FF02003D1
:104E70004FEA835383604FF0005090F84F1011F0C9
:104E8000010101D062B670474EF60022C2F2000264
:104E9000D0F864144FEA114122F8021BD0F86415CF
:104EA0004FEA114122F8021BD0F864164FEA114173
:104EB00022F8021BD0F864174FEA114122F8021BB6
:104EC000D0F864184FEA114122F8021BD0F8641997
:104ED0004FEA114122F8021BD0F8641A4FEA11413F
:104EE00022F8021BD0F8641B4FEA114122F8021B82
:104EF000B0F8901041F20013C2F2000333F801C081
:104F000040F2FF130CEA030C40F6007303EA0103BE
:104F10004FEA03134CEA030C01F00E034FEA03239C
:104F20004CEA030C22F802CB01F1020140F6002307
:104F3000994228BF0021A0F8901090F8921047F2F3
:104F40002803C1F20003082928BF083301F0070C29
:104F50004FEA0C2C6344D3F800C04FEA5C5C40F28B
:104F6000FF730CEA030C4FEAC1234CEA030C22F84E
:104F700002CB01F10101102928BF002180F8921015
:104F800090F8931018291FD247F20003C1F20003D2
:104F9000082928BF0833102928BF083301F0070C5F
:104FA0004FEA0C2C6344D3F800C04FEA5C5C40F23B
:104FB000FF730CEA030C4FEAC1234CEA030C22F8FE
:104FC00002CB01F101011BE040F2A003C2F2000399
:104FD00001F0070C4FEA4C0C6344B3F800C04FEAF1
:104FE0005C0C40F2FF730CEA030C4FEAC1234CEA5D
:104FF000030C22F802CB01F10101202928BF002176
:1050000080F89310B0F8941040F60053C2F20003F9
:1050100013F801C00CF0FF0C4FEA01234CEA030C1B
:1050200022F802CB40F2F8138B4202BF90F8F83E10
:1050300023F0010380F8F83E01F1010140F2002362
:10504000994205D34FF00001B0F8B020A0F8FE2E31
:10505000A0F8941062B6704740F21040C4F200000D
:1050600002684FF00001016012F0010200D17047A8
:105070004FF00050D0F8E42B22F000425FEA3202F9
:105080004FEA9251134681EA030161F39E72C0F820
:10509000E42B704740F60000C4F2000002694FF0B4
:1050A0000001016112F0010200D170474FF0005081
:1050B000D0F8E42A22F000425FEA32024FEA92512D
:1050C000134681EA030161F39E72C0F8E42A704737
:1050D00044F20000C4F2010002694FF0000112F036
:1050E000010200D1704701614FF00050D0F8E4296F
:1050F00022F000425FEA32024FEA9251134681EAFF
:10510000030161F39E72C0F8E429704701617047A2
:1051100044F20040C4F2010002694FF0000112F0B5
:10512000010208D140F20000C4F20100026912F04D
:10513000010202D170470161704701614FF00050D8
:10514000D0F8E42822F000425FEA32024FEA92519E
:10515000134681EA030161F39E72C0F8E4287047A8
:1051600072B641F21040C4F2000002684FF0000134
:10517000016012F0010200D1704746F20042C4F211
:105180000202916D41F0010191654FF000504FF026
:10519000020180F8201162B6704740F60040C4F268
:1051A000000002694FF00001016112F0010200D11C
:1051B000704740F60042C4F2000240F20001C0F223
:1051C000000111604FF000504FF0000180F8B21064
:1051D00090F8F81E41F0020180F8F81E704700BFF9
:1051E0002DE9F04F89B007460C4603924FF00003BB
:1051F000036045F6B06BC0F6020B45F6C063C0F61F
:1052000002030293C2E204F10104252903D12346DB
:105210004FF0000603E0384600F07AFDB6E219468A
:1052200013F8010B1C46A0F12002102A1CD8DFE85D
:1052300002F0091B1B0C1B1B1B0F1B1B1B121B153E
:105240001B1B180046F04006E9E746F08006E6E73B
:1052500046F40046E3E746F02006E0E746F0100695
:10526000DDE746F40076DAE72A2807D0A0F130021D
:10527000D2B2092A13D94FF0000A20E0039B03F1B0
:1052800004000390D3F800A0BAF1000FBCBFCAF12C
:10529000000A46F01006487801F102040FE04FF0D2
:1052A000000A0AEB8A0AA0F1300000EB4A0A13F860
:1052B000010B1C46A0F13002D2B2092AF1D92AEA28
:1052C000EA7A2E282DD120782A2809D004F1010469
:1052D000A0F13003DBB2092B0CD94FF000081DE020
:1052E000039B03F104020392D3F80080607804F179
:1052F000020410E023464FF0000808EB8808A0F1F4
:10530000300000EB480813F8010B1C46A0F13002F6
:10531000D2B2092AF1D9B8F1000F04DB46F4807645
:1053200001E04FF0000868280CD12078682805D1EA
:1053300046F00806607804F1020403E004F1010479
:1053400046F0040678287AD8DFE810F02E027900BB
:105350007900790079007900790079007900790085
:105360007900790079007900790079007900790075
:105370007900790079007900790079007900790065
:105380007900790079007900790079007900790055
:105390007900790079008A00790079007900790034
:1053A0007900790079007900790079007900790035
:1053B0007900790079007900790079007900790025
:1053C0007900790079007900790079007900790015
:1053D0007900790079007900790079007900790005
:1053E00079007900790079007900790079007900F5
:1053F000790079007900790079007900EB00790073
:1054000079007900790079007900790079007900D4
:10541000790090001701790079007900790017016F
:105420007900790079007900AB000001D80079009B
:105430007900B70079000F0179007900ED0040F2A2
:105440000003C2F200031D68002D00F09F81CDF81B
:10545000008003AB0193394632465346A84795E195
:1054600038464FF0250100F053FC8FE1039B03F118
:10547000040203921D780AF1FF3A304651463A463B
:1054800000F074FC3846294600F042FC16F0100F7C
:1054900000F07C814FF0200051463A4600F054FC69
:1054A00074E116F0080F039B03F1040203921B68DA
:1054B0003A6814BF1A701A6068E1039B03F1040292
:1054C0000392D3F80090484600F0A0FC054616F47D
:1054D000807F02D04545A8BF4546C5EB0A0A304645
:1054E00051463A4600F042FC002DCFD019F8011B7E
:1054F000384600F00DFC013DF8D1C7E7039B03F1EE
:10550000040203921B6806F08009B9F1000F14BF72
:105510004FF023094FF0000946F480764FF0080859
:105520006AE046F4005616F0800F07D043F2780385
:1055300043F25809782808BF994601E04FF0000966
:1055400016F4807F20D026F400761DE006F0800956
:10555000B9F1000F14BF4FF030094FF0000916F4F5
:10556000807F11D026F400760EE016F4807F09D0FB
:1055700026F400764FF0000906E046F480464FF02E
:10558000000901E04FF0000916F4804F1ED0039B84
:1055900003F1040203921B6816F0040F01D01BB242
:1055A00003E016F0080F18BFDBB2002B04DAC3F1DA
:1055B00000034FF02D091AE016F0200F15D106F068
:1055C0004002002A18BF4FF0200910E0039B03F1AE
:1055D000040203921B6816F0040F01D09BB206E090
:1055E00016F0080F03D0DBB201E04FF02B0916F4E0
:1055F000807F04D026F4007616F4807F01D14FF02E
:105600000108A0F1580020286FD8DFE800F0196EDB
:105610006E6E6E6E6E6E6E6E6E6E156E6E6E6E155C
:105620006E6E6E6E6E11196E6E6E6E156E6E190068
:105630000BBB4FF000055DE053BB4FF0000559E098
:10564000002B55D04FF0000506F40052DDF808E0BD
:1056500032B103F00F011EF8010005A9685405E0FE
:1056600003F00F011BF8010005A9685405F10105BD
:105670001B09EDD13EE04FF0000503F0070101F1F9
:10568000300105AAA95405F10105DB08F5D131E087
:105690004FF0000506F4004C4CF6CD4ECCF6CC4E47
:1056A0006246A44614465CB105F00302032A07D102
:1056B00008A842194FF02C0102F80C1C05F1010555
:1056C00008AA5119AEFB03024FEAD20202EB820094
:1056D000A3EB400303F1300301F80C3C05F1010595
:1056E0001346002ADFD1644604E04FF0000501E0D4
:1056F0004FF00005C5EB080828EAE878C8EB0A0A6D
:10570000C5EB0A0AB9F1FF0F88BF0AF1FF3AB9F1F8
:10571000000F01D00AF1FF3A16F4007F06D130469F
:1057200051463A4600F022FB4FF0000AB9F1FF0F54
:1057300004D9C9F30721384600F0EAFAB9F1000F9D
:1057400004D05FFA89F1384600F0E2FA304651465B
:105750003A4600F00BFB4FF0300041463A4600F06D
:10576000F3FA012D09D40DF11408454415F8011D73
:10577000384600F0CDFA4545F8D116F0100F05D0A7
:105780004FF0200051463A4600F0DEFA2178002919
:105790007FF439ADBB682BB13A6879688A423CBF67
:1057A00000219954386801E04FF0FF3009B0BDE89E
:1057B000F08F00BF10B504460B783BB1B0F1FF3F4E
:1057C00006D04B6803F1FF334B6001E08B689847CC
:1057D000204610BD2DE9F84F82468B4690469946EB
:1057E0000A9F4FF0FF3500E0354605F101065046AF
:1057F00000F07CFA044600F0FDFA0028F4D1B4F180
:10580000FF3F00F0848028F4C068002F3DDD18F0D1
:10581000800F0FD02B2C03D02D2C09D148F4806899
:1058200005F10206504600F061FA044607F1FF3721
:10583000002F2ADD302C28D148F4007807F1FF37FB
:1058400006F10105504600F051FA0446002F16DD1E
:10585000782801D0582812D1B9F1000F02D0B9F13F
:10586000100F5CD128F4007807F1FF3706F102052C
:10587000504600F03BFA04464FF010094FE0B9F1F2
:10588000000F08BF4FF0080949E0B9F1000F08BF49
:105890004FF00A09002F10DC4FF0000515E048F426
:1058A000007807F1FF3709FB050506F101065046B0
:1058B00000F01CFA044617B907E04FF00005204637
:1058C000494600F079FA0028E9DA20465146FFF708
:1058D00071FF18F4007F1DD018F0010F1CD1DBF808
:1058E000003003F10402CBF800201B6808F490623A
:1058F000B2F5906F08BF6D4218F0100F01D01D7007
:105900000AE018F0080F14BF1D801D6004E04FF07E
:10591000FF3601E06FF001063046BDE8F88F2E46F5
:10592000B8E700BF2DE9F04F87B002908946059295
:105930004FF0000BCDF80CB04CF6CC4AC0F6CC4A78
:105940004C4614F8016B002E00F0CB81252E35D08B
:10595000304600F04FFA08B918E02C4604F1010572
:10596000207800F047FA0028F7D101E00BF1010B95
:10597000029800F0BBF9054600F03CFA0028F5D18A
:1059800028460299FFF716FFA146D9E7029800F0D2
:10599000ADF90546B04203D10BF1010BA146CFE7AB
:1059A0000299FFF707FFB5F1FF3F40F09A81039A94
:1059B000002A08BF4FF0FF32039292E199F80130BC
:1059C0002A2B06BF09F102044FF001084FF000082E
:1059D0004FF000050CE0554500F3838105EB85058C
:1059E000A6F1300616EB450500F17B8148F0200852
:1059F000274604F101043E78A146304600F0D4F970
:105A00000028E8D108F02002002A08BF6FF0004506
:105A10004C2E05D17E7807F1020948F044080EE0CB
:105A2000682E0CD17E78682E05D148F01008BE781B
:105A300007F1030903E007F1020948F00808A6F19D
:105A40002506532E00F24D81DFE816F054004B017D
:105A50004B014B014B014B014B014B014B014B01E6
:105A60004B014B014B014B014B014B014B014B01D6
:105A70004B014B014B014B014B014B014B014B01C6
:105A80004B014B014B014B014B014B014B014B01B6
:105A90004B014B014B014B014B014B014B014B01A6
:105AA0004B014B014B014B014B014B014B014B0196
:105AB0004B012C014B014B014B014B014B014B01A5
:105AC0004B014B014B014B016B009C004B014B0107
:105AD0004B014B01A7004B014B014B014B01B200A5
:105AE000C900D4004B014B01DF004B0121014B01E8
:105AF0004B012C01029800F0F9F80446252802D148
:105B00000BF1010B1CE70299FFF754FEB4F1FF3FC4
:105B100040F0E780039B002B08BF4FF0FF33039357
:105B2000DFE008F02003002B08BF012518F0010476
:105B300005D1059B03F1040205921E6801E04FF0B8
:105B40000006002D00F0CD80002D13DD029800F03E
:105B5000CDF8B0F1FF3F06D1039B002B08BF4FF0FB
:105B6000FF330393BDE00CB906F8010B0BF1010BF9
:105B7000013DEBD1002C7FF4E3AE039B03F1010365
:105B80000393DDE648F080020095029805A94FF0E6
:105B90000A03FFF71FFE04468EE048F080020095DE
:105BA000029805A94FF00003FFF714FE044683E0B6
:105BB00018F0010F7FF4C4AE059B03F104020592B7
:105BC0001B6818F0100F02D083F800B0B8E618F088
:105BD000080F14BFA3F800B0C3F800B0B0E648F057
:105BE00080020095029805A94FF00803FFF7F2FD27
:105BF000044661E028F01E020095029805A94FF0C6
:105C00001003FFF7E7FD044656E04FF0FF3404F1C0
:105C10000104029800F06AF8064600F0EBF800284C
:105C2000F5D1B6F1FF3F2FD018F0010706D1059B43
:105C300003F1040205921B68049302E04FF0000296
:105C40000492002D11DC15E005F1FF351FB9049B0E
:105C500003F8016B049304F10104029800F046F884
:105C600006463DB1B0F1FF3F04D0304600F0C2F827
:105C70000028E9D030460299FFF79CFDE7B94FF0C4
:105C80000002049B1A7017E04FF0FF3414E048F054
:105C900080020095029805A94FF00A03FFF79AFDCC
:105CA000044609E048F080020095029805A94FF0EB
:105CB0001003FFF78FFD0446002C09DAB4F1FF3F13
:105CC0000FD1039A002A08BF4FF0FF32039208E079
:105CD00018F0010F03D1039A02F101020392A344C9
:105CE0002EE6039807B0BDE8F08F00BF08B5034665
:105CF000027832B14268107830B102F101025A6084
:105D000008BD4368984708BD4FF0FF3008BD00BF8D
:105D100038B50446806848B12368626803F101051C
:105D2000954208BF0021934238BFC154E36833B1A4
:105D300020686268904202D208462146984723684C
:105D400003F10103236038BDF8B5154601290BD4D2
:105D50000E464FF00004C7B228463946FFF7D8FF79
:105D600004F10104B442F7D1F8BD00BF08B510F04A
:105D7000100F07D100F4007000280CBF2020302045
:105D8000FFF7E2FF08BD00BFA0F1410019288CBF5A
:105D900000200120704700BFA0F1610019288CBFCE
:105DA00000200120704700BFA0F1300009288CBFFF
:105DB00000200120704700BF38B504460D46FFF7AC
:105DC000F3FF10B1A4F130000FE02046FFF7E4FF2D
:105DD00010B1A4F1570008E02046FFF7D5FF10B13D
:105DE000A4F1370001E04FF0FF30A842A8BF4FF008
:105DF000FF3038BDA0F10903042B04D9202814BFBB
:105E00000020012070474FF00100704700F10101B0
:105E100010F0030F11D010F8012B002A23D010F03E
:105E2000030F0AD010F8012B002A1CD010F0030F2A
:105E300003D010F8012B002A15D02DE970004FF087
:105E400001324FF0803350F8044BA4EB020525EAF1
:105E500004051D4000D1F6E7A0F1040070BC10F865
:105E6000012B002AFBD1A0EB0100704738B5044696
:105E70000D4600F019F840F20403C2F200031D6061
:105E800044F0800440F20803C2F200031C601A468A
:105E90001368002BFCD100F009F840F20403C2F2B1
:105EA0000003186838BD00BF704700BF704700BFCF
:105EB0003031323334353637383961626364656680
:105EC0003031323334353637383941424344454630
:04000005080002BD30
:00000001FF
